:020000040800F2
:10700000A017002099710008997F0008897E000868
:10701000957F0008457A0008798900080000000083
:1070200000000000000000000000000031840008A3
:10703000557C000800000000AF710008B171000825
:10704000B3710008B3710008B37100089982000899
:10705000B3710008B3710008B3710008B371000880
:10706000B3710008B3710008B3710008B371000870
:10707000B3710008B3710008B3710008B371000860
:10708000B3710008B3710008B3710008B371000850
:10709000B3710008B3710008B3710008B371000840
:1070A000B3710008B3710008B3710008B371000830
:1070B000B3710008A5850008B3710008B37100081A
:1070C000B3710008B3710008B3710008B371000810
:1070D000B371000875870008B3710008B371000828
:1070E000B3710008B3710008B371000800F002F832
:1070F00000F042F80AA090E8000C82448344AAF110
:107100000107DA4501D100F037F8AFF2090EBAE80D
:107110000F0013F0010F18BFFB1A43F001031847CB
:107120000880000028800000103A24BF78C878C189
:10713000FAD8520724BF30C830C144BF04680C607D
:10714000704700000023002400250026103A28BFC5
:1071500078C1FBD8520728BF30C148BF0B607047C9
:10716000642900F09D80732900F09B820020704705
:107170001FB51FBD10B510BD00F0D2FA1146FFF7C4
:10718000F7FF03F075FD00F0F0FA03B4FFF7F2FF2C
:1071900003BC00F0F5FA00000948804709480047A1
:1071A000FEE7FEE7FEE7FEE7FEE7FEE7FEE7FEE7B7
:1071B000FEE7FEE704480549054A064B7047000014
:1071C00045850008ED700008A0050020A0170020EC
:1071D000A0070020A00700200FB41CB5074B06AA8B
:1071E0007B4469460090059800F031FA002069461A
:1071F00000F040FA1CBC5DF814FB00009104000094
:1072000070B5044685690068C10601D5302600E0E6
:107210002026C00707D070BDD4E901213046904731
:10722000206A401C20626D1EF6D570BD70B5044604
:1072300085690078C00707D170BDD4E901212020FD
:107240009047206A401C20626D1EF6D570BD70B557
:107250000C460546012A05D02878800600D5EA6943
:10726000002302E0012305E05B1C934202D2E05CB4
:107270000028F9D1A869E618C01AA861286A18443C
:1072800028622846FFF7BCFF04E0D5E9012114F885
:10729000010B9047B442F8D32846FFF7C7FF70BDF3
:1072A0002DE9F0410646002410687529314616A5DF
:1072B00010D0AFF30080002802DA404213A507E0A7
:1072C00031688A0701D512A502E0490704D511A546
:1072D000012401E0AFF3008000210A2206F1240717
:1072E00009E0B0FBF2FCB0FBF2F302FB1C00303013
:1072F00078541846491C0028F3D123462A463046C4
:10730000BDE8F04100F044B9000000002D0000008D
:107310002B000000200000002DE9F0474FF0000A8C
:1073200089460446C0F820A02046E1688847002826
:1073300076D0252806D0D4E901219047206A401C48
:107340002062F1E7E168204600258847C4F81CA0C8
:1073500006460027C4F818A02A2E09D0304601F0AE
:1073600074FB38B304EB8708303EC8F8186019E0A6
:1073700059F8041B204604EB87029161E1688847B5
:10738000012F064618D1E069002820DA25F02005F3
:107390001DE0D8F8180000EB800006EB4000303804
:1073A000C8F818002046E1688847064601F04DFB02
:1073B0000028EED1012F0AD02E2E08D12046E168F8
:1073C00088477F1C0646022F45F02005C4DBA069D4
:1073D000002803DA404245F00105A061E80701D02A
:1073E00025F01005B6B1A6F14100192802D82036C3
:1073F00045F400654A463146204625604D46FFF774
:10740000AFFE58B1012806D0ED1D25F0070000F1B0
:10741000080989E704E005F1040985E730468AE7B1
:10742000206ABDE8F08730B505460B462A4613F8BA
:10743000014B12F8010B08B1A042F8D01CB1002892
:1074400002D06D1CF1E7284630BD40EA010310B5BB
:107450009B070FD1042A0DD310C808C9121F9C42E4
:10746000F8D020BA19BA884201D9012010BD4FF0D6
:10747000FF3010BD1AB1D30703D0521C07E0002023
:1074800010BD10F8013B11F8014B1B1B07D110F880
:10749000013B11F8014B1B1B01D1921EF1D1184683
:1074A00010BD40EA0103024630B59B0710D14FF0F2
:1074B000013400E008C208C91D1B9D4315EAC41F22
:1074C000F8D013F0FF0102F8011B0DD01B0AF8E7FA
:1074D00011F8013B002B02F8013B05D011F8013BEC
:1074E000002B02F8013BF3D130BD032A40F230807B
:1074F00010F0030C00F0158011F8013BBCF1020FF5
:10750000624498BF11F801CB00F8013B38BF11F875
:10751000013BA2F1040298BF00F801CB38BF00F88C
:10752000013B11F0030300F0C080083AC0F008806E
:1075300051F8043B083A51F804CBA0E80810F5E7ED
:10754000121D5CBF51F8043B40F8043BAFF30080D0
:10755000D20724BF11F8013B11F801CB48BF11F845
:10756000012B24BF00F8013B00F801CB48BF00F815
:10757000012B704770477047704710B500F0C8F88E
:10758000006810BD10B5044600F0C2F8046010BDDC
:107590002DE9F0470D4699469246044600F124082D
:1075A0000168880604D5E06921F01001216000E03F
:1075B0000120A84201DD471B00E00027A1697A19DC
:1075C00002EB0900081AA0612078C00602D4204608
:1075D000FFF716FE002608E0D4E901211AF806009C
:1075E0009047206A401C761C20624E45F4DB2078D0
:1075F000C0060AD52046FFF703FE06E0D4E90121C4
:1076000030209047206A401C2062381EA7F10107F5
:10761000F4DC07E0D4E9012118F805009047206A5E
:10762000401C2062281EA5F10105F3DC2046FFF76F
:10763000FDFD2078000602D50220BDE8F08701207C
:10764000FBE7000001694A1C02610878704700B539
:107650008FB0CDE901310021059105497944CDE98B
:10766000031011466846FFF757FE0FB000BD00003B
:10767000E5FFFFFF0A6802F8010B0A60704710B5CA
:10768000436913B1AFF3008001E0FFF7E0FD012093
:1076900010BD127800F124010A7000224A70012204
:1076A000EDE711684FF0FF32E9E710B5203AC0F07E
:1076B0000B80B1E81850203AA0E81850B1E81850F3
:1076C000A0E81850BFF4F5AF5FEA027C24BFB1E830
:1076D0001850A0E8185044BF18C918C0BDE81040A1
:1076E0005FEA827C24BF51F8043B40F8043B08BFAA
:1076F0007047D20728BF31F8023B48BF11F8012B71
:1077000028BF20F8023B48BF00F8012B704700005B
:1077100000487047400500200048704740050020A1
:107720007546FFF7F9FFAE4605006946534620F05F
:107730000700854618B020B5FFF73CFDBDE82040A6
:107740004FF000064FF000074FF000084FF0000B1D
:1077500021F00701AC46ACE8C009ACE8C009ACE8D0
:10776000C009ACE8C0098D46704710B50446AFF3B8
:1077700000802046BDE81040FFF707BD70470000BD
:1077800001491820ABBEFEE72600020000B585B017
:107790004FF4004000F050FC1E4800F053F8002069
:1077A000009001208DF804008DF805004FF4602052
:1077B00002900020039002208DF8100069461548C1
:1077C00000F082F8072301220221124800F0A4F8F9
:1077D0000723022205210F4800F09EF801210D48E1
:1077E00000F025F801210B4800F016F8094800F0D8
:1077F000EFF800BF074800F05DF80028FAD105480F
:1078000000F0F6F800BF034800F04AF80028FAD16B
:1078100005B000BD0024014021B1826842F00102A0
:10782000826003E0826822F001028260704721B129
:10783000826842F48072826003E0826822F480727F
:107840008260704710B504461248844208D1012175
:10785000401500F02DFC0021601500F029FC17E018
:107860000D48844208D10121001500F021FC0021BF
:10787000201500F01DFC0BE00848844208D10121CE
:10788000C80300F015FC00214FF4004000F010FC8C
:1078900010BD00000024014000280140003C0140D0
:1078A000014600208A6802F004020AB1012000E0CB
:1078B00000207047014600208A6802F008020AB1E1
:1078C000012000E00020704730B502460020002370
:1078D00050680F4C20400D790C6844EA0524204381
:1078E000506090680B4C2040D1E902542C434D79F4
:1078F00044EA450420439060D06A20F470000C7C78
:10790000641EE4B2234340EA0350D06230BD00005D
:10791000FFFEF0FFFDF7F1FFF0B504460D46002035
:107920000021092D11DDE068A5F10A0606EB4607E6
:10793000072606FA07F18843A5F10A0606EB460674
:1079400003FA06F10843E0600CE0206905EB450707
:10795000072606FA07F1884305EB450603FA06F108
:1079600008432061072A0FDA606B561E06EB860774
:107970001F2606FA07F18843561E06EB860605FA0F
:1079800006F10843606322E00D2A0FDA206BD61F50
:1079900006EB86071F2606FA07F18843D61F06EB7B
:1079A000860605FA06F10843206310E0E06AA2F1BA
:1079B0000D0606EB86071F2606FA07F18843A2F19B
:1079C0000D0606EB860605FA06F10843E062F0BDF7
:1079D000816841F008018160704721B1826842F4FA
:1079E000A002826003E0826822F4A00282607047F5
:1079F000816841F004018160704710B5012000F0FA
:107A000067FB002000F064FB10BD000008B50146D4
:107A100000200090034800900098084400900098CF
:107A2000008808BD006C004008B500220092044A9E
:107A30000092009A02440092009A116008BD000072
:107A4000006C004000BFFEE7014601EBC1000522CB
:107A500090FBF2F000F5A07080B2704721B102688F
:107A600042F00102026004E002684FF6FE731A4021
:107A70000260704700B58BB00121084600F0E8FABB
:107A80000F4800F023F80F4800900F4801900020A5
:107A90000290142003900020049080200590400064
:107AA0000690800007902020089000020990002096
:107AB0000A906946024800F0AFF80BB000BD000024
:107AC000080002404C2401406804002001684FF681
:107AD000FE72114001600021016041608160C1605F
:107AE0004B49884208D14A490839496841F00F0199
:107AF000474A083A51608AE045491431884208D122
:107B000043490839496841F0F001414A083A516057
:107B10007DE03F492831884208D13D49083949680C
:107B200041F470613A4A083A516070E038493C319A
:107B3000884208D136490839496841F47041344ACD
:107B4000083A516063E032495031884208D13049E7
:107B50000839496841F470212D4A083A516056E0CD
:107B60002B496431884208D129490839496841F4D0
:107B70007001274A083A516049E025497831884226
:107B800008D123490839496841F07061204A083A10
:107B900051603CE01F49884206D1011F096841F04D
:107BA0000F01021F116032E01A491431884208D1D6
:107BB0001849091F096841F0F001164A121F1160A7
:107BC00025E014492831884208D11249091F096863
:107BD00041F470610F4A121F116018E00D493C31E9
:107BE000884208D10B49091F096841F47041094ACC
:107BF000121F11600BE007495031884207D1054937
:107C0000091F096841F47021024A121F1160704770
:107C1000080002400804024010B50022026847F63E
:107C2000F0739A430C6A8B6823430C6923434C69B5
:107C300023438C692343CC6923434C6A23438C6AD6
:107C400023431A430260CB6843600B6883604B6830
:107C5000C36010BD70470146A1F5A07202EB82021D
:107C600090B2092290FBF2F290B270472DE9F041F8
:107C7000024600250026002000230024002791F85A
:107C800003C00CF00F0591F803C00CF0100CBCF110
:107C9000000F03D091F802C04CEA050591F800C02E
:107CA000BCF1000F31D0146800202BE04FF0010C24
:107CB0000CFA00F3B1F800C00CEA03069E4220D192
:107CC00083004FF00F0C0CFA03F7BC4305FA03FCDA
:107CD0004CEA040491F803C0BCF1280F06D14FF020
:107CE000010C0CFA00FCC2F814C00AE091F803C0C1
:107CF000BCF1480F05D14FF0010C0CFA00FCC2F8A2
:107D000010C0401C0828D1D31460B1F800C0BCF1E9
:107D1000FF0F34DD546800202EE000F1080C4FF016
:107D2000010808FA0CF3B1F800C00CEA03069E4201
:107D300021D183004FF00F0C0CFA03F7BC4305FA76
:107D400003FC4CEA040491F803C0BCF1280F05D1F0
:107D500000F1080C08FA0CF8C2F8148091F803C07E
:107D6000BCF1480F07D100F1080C4FF0010808FAE8
:107D70000CF8C2F81080401C0828CED35460BDE82F
:107D8000F0810000F0B50A46002300240021002500
:107D900000F00046B6F1004F02D11D4EF16901E03E
:107DA0001B4E7168C0F3034583B200F44016B6F56C
:107DB000401F08D121F07061154E766826F070667C
:107DC000134F7E6012E000F48016B6F5801F06D1D6
:107DD000032606FA05F4A14341F0706106E0460D62
:107DE000360103FA06F6B14341F0706122B1460D47
:107DF000360103FA06F6314300F00046B6F1004FB3
:107E000002D1034EF16101E0014E7160F0BD00004E
:107E1000000001400246002093680B400BB1012096
:107E200000E0002070470146C86880B270470246F3
:107E30000020D3680B400BB1012000E00020704708
:107E40004161704701617047C160704770B502467B
:107E50000D46FF21FF23002409E012F8010B80EA00
:107E600001040748005D80EA03010648035D281EFF
:107E7000A5F10106B5B2F0D143EA012070BD0000C2
:107E8000D6EE0008D6EF000800BFFEE710B502F0FE
:107E9000F7FB4FF480710F48FFF7D4FF40210E48E5
:107EA000FFF7D0FF02210C48FFF7CCFF4FF4007121
:107EB0000848FFF7C5FF4FF47A7001F041F94FF41D
:107EC00000710448FFF7BEFF4FF4FA7001F038F973
:107ED00010BD0000000C01400008014070B50446D0
:107EE0004FF400511148FFF7ABFF02F021FB10489F
:107EF000FFF799FF00F47F4040EA040529460C484B
:107F0000FFF7A2FF4FF480710948FFF799FF0221A4
:107F10000848FFF795FF02210648FFF793FF4FF44B
:107F200080710348FFF78EFF70BD00000010014014
:107F3000000C01400008014070B504464FF40051A8
:107F40001148FFF77FFF02F0F3FA1048FFF76BFFCD
:107F500000F47F4040EA040529460C48FFF774FF0F
:107F60004FF480710948FFF76BFF02210848FFF7C3
:107F700067FF02210648FFF765FF4FF48071034851
:107F8000FFF760FF70BD000000100140000C0140D1
:107F90000008014000BFFEE7704710B54FF4A06035
:107FA00000F03AF810BD000070B5002100230F2248
:107FB000C47804B3154C246804F4E064C4F5E064A8
:107FC000210AC1F10403CA40447804FA03F1847819
:107FD0001440214309010E4C0678A155047804F0A1
:107FE0001F050124AC4005786D11AD0005F1E025B9
:107FF000C5F8004109E0047804F01F050124AC40F5
:10800000044D0678761145F8264070BD0CED00E071
:1080100000E400E080E100E002490143024A11600F
:10802000704700000000FA050CED00E0014908620D
:108030007047000000000E4201460020034A5068CD
:1080400020F4404008435060704700000010024098
:1080500029B1064A52690243044B5A6104E0034ABB
:1080600052698243014B5A61704700000010024080
:1080700029B1064AD2690243044BDA6104E0034A9B
:10808000D2698243014BDA61704700000010024060
:1080900029B1064A92690243044B9A6104E0034AFB
:1080A00092698243014B9A617047000000100240C0
:1080B00029B1064AD2680243044BDA6004E0034A5D
:1080C000D2688243014BDA60704700000010024022
:1080D00001490860704700004004424230B5002169
:1080E0000022002400232D4D6D6805F00C0121B104
:1080F000042905D0082923D105E0294D056022E097
:10810000274D05601FE0254D6D6805F47012234D65
:108110006D6805F48034022505EB92421CB9214DAF
:10812000554305600BE01D4D6D6805F400351DB12C
:108130001C4D5543056002E0194D5543056002E0B2
:10814000174D056000BF00BF144D6D6805F0F001CC
:108150000909154D6B5C0568DD4045600F4D6D6884
:1081600005F4E061090A104D6B5C4568DD408560EF
:108170000A4D6D6805F46051C90A0B4D6B5C45688A
:10818000DD40C560054D6D6805F44041890B074D24
:108190006B5CC568B5FBF3F5056130BD00100240AE
:1081A00000127A0000093D000A0000201A00002099
:1081B00010B501460022002300204A11012A02D1F5
:1081C000094C236806E0022A02D1074C236A01E029
:1081D000054C636A01F01F02012494401C400CB15D
:1081E000012000E0002010BD0010024000210B4AD9
:1081F00011700A4A203A82F82010012802D004287F
:1082000008D103E00121054A117004E00521034A69
:10821000117000E000BF00BF704700002010024056
:1082200001490860704700003C0442420249096A63
:108230000143014A11627047001002400249098857
:108240008143014A11807047042800400348008898
:1082500040F01000014908807047000004280040E9
:10826000034800884FF6EF710840014908807047C5
:108270000428004001460020064A12880A40D0B275
:10828000044A121F12880A4012B108B1012000E00E
:10829000002070470428004010B50120FFF7EAFFD6
:1082A000002866D002F03EFF38480068010C0C2020
:1082B000FFF7BAFB3548008881B21020FFF7B4FB06
:1082C000334801881420FFF7AFFB4FF400613148B9
:1082D000FFF7ADFD20B101211820FFF7A5FB03E05A
:1082E00000211820FFF7A0FB2948008820B128486A
:1082F0000088401E264908802748007820B126487B
:108300000078401E244908702448007820B1234892
:108310000078401E214908702148007820B120488B
:108320000078401E1E4908701E48007820B11D4884
:108330000078401E1B4908701B48008828B11A4865
:108340000088401E1849088013E01848C07A0128A8
:108350000FD181020F48FFF76AFD50B11448007831
:1083600038B91448007820B94FF480610948FFF704
:1083700067FD0220FFF77EFF10B10220FFF75EFFCE
:108380000520FFF75BFF00F037F810BD7C000020F0
:1083900072000020000C0140840000203300002007
:1083A0006C0000208500002082000020FA040020DC
:1083B0006F0000207000002029B1064A1288024395
:1083C000044B1A8004E0034A12888243014B1A804E
:1083D000704700000028004000B50246FFF736FF56
:1083E000C2F3034003490880091D0A80FFF738FFE4
:1083F00000BD00000828004000BF0348008800F0CE
:1084000020000028F9D07047042800400748008861
:108410004FF6F77108400549088000BF03480088FF
:1084200000F008000028F9D0704700000428004040
:10843000704710B500F002F810BD00000CB5002028
:10844000019000903348006840F480303149086062
:1084500000BF3048006800F4003000900198401CD4
:108460000190009820B94FF6FF7101988842F0D131
:108470002848006800F4003010B10120009001E0AD
:10848000002000900098012843D12348006840F064
:108490001000214908600846006820F003000860C9
:1084A0000846006840F0020008601A484068194910
:1084B00048600846406848600846406840F480606C
:1084C00048600846406820F47C10486008464068D0
:1084D00040F4F81048600846006840F0807008607A
:1084E00000BF0C48006800F000700028F9D009486F
:1084F000406820F00300074948600846406840F0A3
:108500000200486000BF0348406800F00C000828E3
:10851000F9D10CBD0010024000200240042808D10F
:108520004FF0E021096941F004014FF0E0221161B0
:1085300007E04FF0E021096921F004014FF0E0224B
:108540001161704710B51248006840F001001049F1
:108550000860084640680F4908400D4948600846D1
:1085600000680D4908400A4908600846006820F480
:10857000802008600846406820F4FE0048604FF400
:108580001F008860FFF755FF04480549086010BDCB
:10859000001002400000FFF8FFFFF6FE0070000828
:1085A00008ED00E010B50121164800F076F808B398
:1085B0000121144800F062F80120134908701348A3
:1085C00000780A2805DA11480078401C0F49087025
:1085D00017E002F06FFE00200C49087001200C49E2
:1085E00008700C480078322805DA0A480078401CE8
:1085F0000849087005E00020064908700120064976
:10860000087010BD0004004022000020250000205A
:108610002300002026000020240000207FB505460E
:108620000C4601210220FFF723FDADF80850ADF8FC
:1086300004400020ADF80A00ADF8060001A90E487C
:1086400000F046F8012211460B4800F037F81D20D3
:108650008DF8000001208DF8010003208DF8020044
:1086600001208DF803006846FFF79EFC01210248B7
:1086700000F007F87FBD000000040040CA430282FA
:10868000704721B1028842F00102028004E00288B2
:108690004FF6FE731A400280704730B50246002044
:1086A00000230024158A05EA0103958905EA0104DF
:1086B00013B10CB1012000E0002030BD1AB1838954
:1086C0000B43838102E083898B43838170470000E1
:1086D000002202881D4B98420ED01D4B98420BD0B1
:1086E000B0F1804F08D01B4B984205D01A4B9842EE
:1086F00002D01A4B984204D14FF68F731A404B8820
:108700001A43174B984207D0164B984204D04FF6A5
:10871000FF431A40CB881A4302808B8883850B88DD
:1087200003850A4B98420BD0094B984208D00E4B58
:10873000984205D00D4B984202D00D4B984201D182
:108740000B7A03860123838270470000002C0140CE
:10875000003401400004004000080040000C0040CC
:10876000001000400014004000400140004401405F
:108770000048014010B520211F4800F05EF8012894
:1087800015D11E480078C82802DB00201B4908705C
:108790001949091D0988CAB218490878411C174BA4
:1087A000197017490A5400201649087023E0402127
:1087B000114800F042F801281DD140210E4800F078
:1087C00027F80E4800781049097888420ADA0B49E0
:1087D0000878411C094A11700949095C064A121DB2
:1087E000118008E080210948FFF72AFB0020034997
:1087F00008700549087010BD0038014028000020AD
:10880000A0030020270000202900002000080140CC
:1088100001F40072B2F5007F00D100BFCA430280AC
:10882000704721B1828942F40052828104E082893A
:108830004DF6FF731A408281704702460020B1F561
:10884000007F00D100BF13880B400BB1012000E076
:1088500000207047F0B503460024002600250020C4
:1088600040F66A17B94200D100BF1846C1F342145E
:1088700001F01F06012707FA06F5012C01D10C3083
:1088800004E0022C01D1103000E014301AB1076866
:108890002F43076002E00768AF430760F0BD0000A8
:1088A0002DE9F04786B005460E460024A24600BFDB
:1088B000A1460027B08900B100BF2F462C8A4CF694
:1088C000FF700440F08804432C82AC894EF6F3100C
:1088D0000440B08831890843718908430443AC815E
:1088E000AC8A4FF6FF400440B0890443AC8201A833
:1088F000FFF7F4FB1F48874202D1DDF810A001E02A
:10890000DDF80CA0A88900F4004040B10AEBCA00D1
:1089100000EB0A1031684900B0FBF1F807E00AEB00
:10892000CA0000EB0A1031688900B0FBF1F864203E
:10893000B8FBF0F004012009642101FB1089A8892B
:1089400000F4004040B1322000EBC900B0FBF1F070
:1089500000F00700044308E0322000EB0910642116
:10896000B0FBF1F000F00F0004432C8106B0BDE82D
:10897000F08700000038014000BFFEE72DE9F0411C
:108980004F1E00EBC7010446D1E9000115461E4603
:1089900037F006020DD02A46334603F0DFFB7F1E78
:1089A00004EBC703D3E9002303F02EF937F00602E6
:1089B000F1D1022F25D0042F13D0062F18BFBDE808
:1089C000F0812A46334603F0C9FBD4E90A2303F0B9
:1089D0001BF92A46334603F0C1FBD4E9082303F010
:1089E00013F92A46334603F0B9FBD4E9062303F012
:1089F0000BF92A46334603F0B1FBD4E9042303F014
:108A000003F92A46334603F0A9FBD4E9022303F015
:108A1000FBF82A46334603F0A1FBD4E90023BDE866
:108A2000F04103F0F1B8000000221346104601495E
:108A300003F0A6B90000F03F012203F0B5BD00220B
:108A400013461046114603F09BB930380A2801D26C
:108A5000012070470020704710B50022002014E06C
:108A6000002107E00A4B03EB810333F810301A446E
:108A70004B1CD9B20A29F5DB0A23B2FBF3F3054CF0
:108A800024F810300022431CD8B20228E8DB10BDC5
:108A9000680400202A00002008B501214802FFF7E1
:108AA000F7FA48208DF803000420ADF8000069466D
:108AB0000C48FFF7DBF800208DF803002020ADF80C
:108AC000000069460748FFF7D1F8FEF75FFEFEF7A2
:108AD000D1FF01210448FEF780FF01210348FEF782
:108AE000BDFF08BD0008014000240140080002400D
:108AF0002DE9F0410446002500264FF6FF77AC46ED
:108B00000FE0208805443AB12088B04200DD268875
:108B10002088B84200DA2788A41C0CF101001FFA53
:108B200080FC8C45EDDBF01BC82802DD01201870AD
:108B300001E00020187042B1A81BA0EB0708881EB6
:108B4000B8FBF0F080B2BDE8F081B5FBF1F080B287
:108B5000F9E700002DE9F04F8BB056480078132854
:108B600005DA54480078401C5249087002E00020A1
:108B70005049087001F0ECF94F494E4A127821F83B
:108B800012000AAB012214214B48FFF7B1FF8246C5
:108B90004FF4FA500AFB00F0CAF58051B0FBF1FB2C
:108BA000584603F0C7FACDE9000101F0B3FECDE964
:108BB00002010020414901F0ADFE8046DDE90223BB
:108BC00003F0D6FB00223E4BCDE9040103F0C6FAC8
:108BD00000223C4BCDE9060103F0BEFB06463246BF
:108BE0000B460020384903F0CBF804460022374BEF
:108BF00003F0BEFBCDE9080103F056FA00B2344998
:108C000008800846B0F9000010F1C80F08DB0846DC
:108C1000B0F90000B0F5487F02DC9DF8280018B1DB
:108C200001202C49087002E000202A4908702849D8
:108C3000098888B2FEF708FF00B2274908800120A2
:108C4000244908700846007830BB24480078022880
:108C50000AD12348007838B91F480078214909789B
:108C6000401A40B2204908701C48007830B11B48B7
:108C7000007802280BD11A48007840B116480088C5
:108C8000194991F90010401A1849088008E0154860
:108C900000881649088003E01248008813490880BC
:108CA00012480088FEF7D7FF114908800BB0BDE8D5
:108CB000F08F000057000020900400200088C3407F
:108CC00000A0724000DCAE408F7366410054A540A6
:108CD0005000002055000020520000205E000020BF
:108CE0005600002066000020540000206400002090
:108CF000620000202DE9F04385B004460B34A778CC
:108D0000E07840EA07272579607940EA05250B3CA1
:108D10000C22B2492046FEF798FB002878D10B348C
:108D20006078102875D1C82FFCD14FF000084FF0A3
:108D300002090020AA490880AA48C07A012817D150
:108D4000C102A948FFF773F8F8B1A848007838B114
:108D5000A348008820F00100401CA149088022E0BF
:108D60009F48008820F00200801C9D4908801AE07E
:108D70004FF400619C48FFF75AF838B198480088D2
:108D800020F00100401C964908800CE04FF48061FF
:108D90009548FFF74CF830B19148008820F0020068
:108DA000801C8F4908804FF480719148FFF73FF88D
:108DB00020B908218E48FFF73AF830B1884800887A
:108DC00020F00400001D8649088010218848FFF724
:108DD0002EF830B18248008820F008000830804921
:108DE00008808048C17A7E48008861F305107C497C
:108DF00008807E48007810B97E48007850B17848E5
:108E0000008820F4004000F500407549088007E024
:108E10009CE0D1E07248008820F40040704908804E
:108E2000754800887549097808446D49098860F3D8
:108E30008E116B48018000880012ADF80000684870
:108E40000088ADF80200072D04D04FF003084FF062
:108E5000010969E0E579207A40EA0525684805803E
:108E60004FF6FF70854206D15E48407A18B901205E
:108E70006449087002E0002062490870657AA07AAF
:108E800040EA052557484580E57A207B40EA0525DC
:108E900054488580657BA07B40EA052551498D714A
:108EA000E57B207C40EA05250D72657CA07C40EACC
:108EB0000525CD71E57C207D40EA05254D724FF0FA
:108EC00002090846407A02280FD140F28A204C4914
:108ED0000880444880790988A1EB4000401E414940
:108EE000488008464088888012E03E48407A03283F
:108EF0000ED140F28A20424908803A488079098898
:108F000001EB4000401C3749488008464088888073
:108F100034494888FEF79FFE3B49088031498888DC
:108F2000FEF799FE394908800B3C43464A4669469C
:108F3000204601F07DFF0546284602F0CFF80020CC
:108F40003349087002203349087044E0002606E0E7
:108F5000A05D10B105B0BDE8F083701CC6B20C2E48
:108F6000F6DB0B346078042835D1642F33D1012D22
:108F700031D12948007800B32648007801281CD157
:108F800026480078C8B10020234908708046072091
:108F9000ADF800000B3C1148016821604168616038
:108FA0008068A060434601226946204601F040FFE8
:108FB0000546284602F092F80DE01648007818B9E8
:108FC00001201449087006E012480078012802D1F7
:108FD00000200F49087000BFBCE700001E050020FC
:108FE00088000020FA040020000C01406F000020DF
:108FF0000008014070000020720000208500002061
:109000006600002056000020680000206A00002052
:109010005F0000205E00002030000020760000206D
:1090200010B590B01348006801901248001D006808
:1090300002901048083000680390002409E00E49AF
:1090400001EB4400B0F8E80F0AA921F81400601CF5
:10905000C4B20C2CF3DB04A901A800F00FF818220D
:1090600004A90AA8FEF7F1F910B9012010B010BD4B
:109070000020FBE7E8F7FF1F0060000818B500229A
:10908000009211E002780B4B9DF800401A5510F841
:10909000012B01F8012B9DF8002001F8012B9DF810
:1090A0000020521CD2B200929DF800200C2AE9DB6D
:1090B00018BD00001E05002010B504466FF0040026
:1090C000FFF72CFAE11704EB5171C1F3C701074A0E
:1090D00011701046007800EB4001C1EBC0104FF654
:1090E000FF7101EAC0000249088010BD1E00002087
:1090F000200000200146114A12884A434FF0E02325
:109100005A6100229A611A46126942F001021A61FC
:1091100000BF4FF0E022106900F001021AB100F424
:109120008032002AF5D04FF0E022126922F00102CD
:109130004FF0E0231A6100229A617047200000205E
:1091400000BF411E88B20028FBD170470146114A7A
:1091500012784A434FF0E0235A6100229A611A467E
:10916000126942F001021A6100BF4FF0E02210695B
:1091700000F001021AB100F48032002AF5D04FF05D
:10918000E022126922F001024FF0E0231A6100226E
:109190009A6170471E00002010B500F029F80120E8
:1091A00001F008FA01242246641C0B48007804FBF5
:1091B0000020C1B209A2272001F088FB2246641CCE
:1091C0000548007804FB0020C1B205A2032001F08D
:1091D0007DFB02F0A3FC10BD090000204D435500AB
:1091E000446576696365204944204572726F720058
:1091F00000200021084A00BF0BE0002004E000230B
:1092000002F8013B431CD8B26028F8DB01F10803E7
:10921000D9B24029F1DB7047A00000201CB5FFF750
:10922000E7FF022001F0C6F912A20421084601F06E
:109230004DFB13A21421042001F048FB1348C08900
:109240003C2190FBF1F4224611A11348FDF7C4FF25
:10925000114A2A21202001F039FB022003213A2360
:109260004C22CDE900102821182002F029FC02F040
:1092700055FC1CBD20486F7420537461727400004B
:1092800020202044656C617900000000FA04002071
:1092900025646D696E7300002A0500207CB5FFF718
:1092A000A7FF052001F086F9F9480078022803D0CD
:1092B000F848007800286ED1F548007801286AD077
:1092C000F54840880028FAD0F348407A012805D1B3
:1092D000F2A21421182001F0F9FA45E2EE48407A92
:1092E000022803D0EC48407A032805D1ECA21421CF
:1092F000202001F0EBFAECE0E748C07900287CD0B0
:10930000E548007A10B1E448448801E0E2488488E6
:109310000A20B4FBF0F63246E2A1E348FDF75CFF19
:10932000B4F57A7F05D3E04A0821182001F0CEFA7F
:1093300004E0DD4A0821242001F0C8FADB48008857
:109340004FF6FF71884204D1D9A1D748FDF744FFF9
:1093500009E0D64800880A2190FBF1F63246D1A1F7
:10936000D148FDF739FFD1480088B0F57A7F05DB99
:10937000CD4A2221182001F0A9FA04E0CA4A22218C
:10938000242001F0A3FA012001F014F9B4F57A7F4A
:1093900002D3042501E0C9E1002505F14401C8B26A
:1093A000C4A2102101F092FA0120009005F14201BF
:1093B000CAB2491E0190C8B21123102102F080FBED
:1093C000BA480088B0F57A7F01DB042500E000256B
:1093D00005F14401C8B2B7A22A2101F077FA0120B1
:1093E000009005F14201CAB2491E0190C8B22B2378
:1093F0002A2102F065FB62E0FFE7A748007A10B17E
:10940000AD48048801E0AD4804880A20B4FBF0F6BA
:109410003246A4A1A448FDF7DFFEB4F57A7F05D358
:10942000A14A0821182001F051FA04E09E4A0821BF
:10943000242001F04BFA9D4800884FF6FF718842C6
:1094400004D19BA19848FDF7C7FE09E09C4800881D
:109450000A2190FBF1F6324692A19348FDF7BCFE3B
:1094600092480088B0F57A7F05DB8F4A22211820C8
:1094700001F02CFA04E08C4A2221242001F026FA83
:10948000012001F097F88FA21021442001F01EFA6C
:10949000012000901123422210210190412002F06E
:1094A0000FFB88A22A21442001F010FA012000902D
:1094B0002B2342222A210190412002F001FB82A2AB
:1094C00000211C2001F002FA82A23821202001F0A4
:1094D000FDF9012001F06EF86E480078D0B96C48B3
:1094E000007830B16A480078022813D17B480078B0
:1094F00080B17B48007848B17A4A0021522000F0C0
:10950000B9FF79A20A215A2001F0E0F90120774938
:10951000087002E000207549087075480078E0B3D3
:109520005D48C07A01280AD1C1027248FEF77FFC6B
:1095300028B97148008810B16948007878B94FF4AB
:1095400000616C48FEF773FC48B95348C07A0128A3
:1095500031D04FF480616748FEF769FCE8B167A23B
:109560001821002001F0B2F966A22221062001F0A4
:10957000ADF908216448FEF75AFC50B963480078F9
:1095800000285AD062480078002856D05448007805
:10959000F0B355A23021082000E00CE001F096F96C
:1095A000032001213A231022CDE900102D210420AF
:1095B00002F086FA41E05748007848B34FF4006162
:1095C0004C48FEF734FC40B94B48008810B952486B
:1095D000007810B14248007828B94FF4006145483E
:1095E000FEF725FCA0B14DA21821002001F06EF974
:1095F00044A22221062001F069F94FF4807142480B
:10960000FEF715FC50B94148007808B1404800E029
:1096100013E0007888B13248007870B132A230216E
:10962000082001F053F9032001213A231022CDE94B
:1096300000102D21042002F043FA1748807A90B1DF
:1096400030A21C21542001F041F91348407AE8B9B6
:109650000120032121234C22CDE900101F211A20D3
:1096600002F02EFA80E02FA21C21482001F02EF9F2
:109670000948407A50B90120032121234422CDE931
:1096800000101F211A2002F01BFA6DE06CE00000B0
:109690005E00002055000020FA0400204F464600DE
:1096A0004F4E0000253264002A050020640000208F
:1096B0002D2D2D0046000000680000206A000020CB
:1096C0006200002043000000536574706F696E747F
:1096D0000000000043757272656E74005600002031
:1096E0006E000020C4EE000832000000740000206C
:1096F00070000020000C0140720000204865617479
:10970000000000004F6E0000000801406D000020C6
:109710006C0000206F00002075000020436F6F6C0C
:10972000000000004175746F0000000015480078CB
:1097300090B1022000F03EFF13A20021084601F084
:10974000C5F815A21421002001F0C0F815A22821A7
:10975000042001F0BBF807E0022000F02BFF13A269
:109760001821042001F0B2F81348007838B1012024
:1097700000F020FF11A20021084601F0A7F802F036
:10978000CDF97CBD5E000020506C65617365207072
:109790007265737300000000204164647265737326
:1097A000696E6700202020204B65790020204F66DD
:1097B000666C696E650000004F0000206565707280
:1097C000000000001CB5FFF713FD022000F0F2FEC0
:1097D00015A20421002001F079F816A2142100201E
:1097E00001F074F81648427B16A11748FDF7F4FC07
:1097F0001348407B0A2805DB134A2A21242001F064
:1098000065F804E0104A2A21282001F05FF80220C0
:1098100003213A233C22CDE900102821222002F026
:109820004FF902F07BF91CBD20436F6D70726573B8
:10983000736F72002064656C61792074696D6500D6
:10984000FA040020256473002A05002010B5FFF7F4
:10985000CFFC022000F0AEFE0AA20A21002001F097
:1098600035F8012000F0A6FE0AA22321042001F011
:109870002DF80CA23221042001F028F802F04EF954
:1098800010BD000052657365742053797374656D63
:10989000000000004144445220746F20636F6E66E4
:1098A00069726D00202046414E20746F2062616312
:1098B0006B00000010B5FFF79BFC022000F07AFE61
:1098C0000AA20821002001F001F80CA21C210020AE
:1098D00000F0FCFF012000F06DFE0BA23221002001
:1098E00000F0F4FF02F01AF910BD00005265736534
:1098F000742053797374656D0000000020202020CF
:10990000446F6E650000000020506C656173652037
:10991000526573746172740010B5FFF769FC4348B7
:10992000C07A00281FD1022000F044FE40A2052189
:10993000042000F0CBFF012000F03CFE3FA21921E3
:10994000032000F0C3FF41A22321002000F0BEFF4E
:1099500043A22D21002000F0B9FF46A237210320A9
:1099600000F0B4FF5FE03148C07A03281AD102202A
:1099700000F020FE43A20521042000F0A7FF0120F3
:1099800000F018FE42A21921032000F09FFF44A21C
:109990002321002000F09AFF45A22D21002000F095
:1099A00095FF40E02148C07A022819D100F002FE5C
:1099B00042A20521042000F089FF012000F0FAFDF9
:1099C00041A21921002000F081FF43A2232103209E
:1099D00000F07CFF36A22D21002000F077FF22E06E
:1099E0001248C07A01281ED1022000F0E3FD3EA2F9
:1099F0000521042000F06AFF012000F0DBFD0FA22A
:109A00001921032000F062FF3AA22321002000F078
:109A10005DFF13A22D21002000F058FF39A237214D
:109A2000032000F053FF02F079F810BDFA04002083
:109A300020486561742F436F6F6C0000576974682C
:109A4000206F7220776974686F7574004D756C743F
:109A500069706C65207374616765732E0000000087
:109A600041646A75737420627920776972696E67E0
:109A700000000000202020572C57322C592C59323E
:109A80000000000020436F6F6C206F6E6C79000047
:109A9000202043656E7472616C2061697200000061
:109AA0002020636F6E646974696F6E696E67000071
:109AB0002020202020206F6E6C79000020486561F6
:109AC00074206F6E6C7900002020204761732C6F2A
:109AD000696C206F7200000020656C6563747269A8
:109AE00063206865617400002048656174207075AA
:109AF0006D70000020617578696C69617279206809
:109B00006561740020202020204155582F45000019
:109B100010B5FFF76DFB1E48007B00281AD002200D
:109B200000F048FD1BA20A21042000F0CFFE012016
:109B300000F040FD1AA21E21002000F0C7FE1CA26A
:109B40002821002000F0C2FE1EA23221002000F0D9
:109B5000BDFE19E0022000F02DFD1FA20A21042005
:109B600000F0B4FE012000F025FD0DA21E21002012
:109B700000F0ACFE1BA22821002000F0A7FE11A2DD
:109B80003221002000F0A2FE01F0C8FF10BD00004D
:109B9000FA0400202020436F6F6C696E670000009C
:109BA00020412077697265206C6162656C65640094
:109BB000224F2220636F6E6E656374656420746F3C
:109BC00000000000746865204F2F42207465726D9C
:109BD000696E616C00000000202048656174696E48
:109BE0006700000022422220636F6E6E6563746519
:109BF0006420746F0000000010B5FFF7F9FA02202E
:109C000000F0D8FC084A0A21202000F05FFE074A35
:109C100007A10948FDF7E0FA074A1E21042000F0D9
:109C200055FE01F07BFF10BDEA040020E004002097
:109C300020202056202573002A05002008B5012188
:109C40000420FEF725FA03208DF8020010208DF87D
:109C50000300C001ADF8000069460848FEF706F8A9
:109C60004FF48050ADF8000014208DF803006946D1
:109C70000248FDF7FBFF00F0B2F908BD0008014003
:109C80002DE9F04707460C4690461D46DDF820902A
:109C900000260AE000F010FA384600F0D1F900B9C9
:109CA00005E000F014FA701CC6B2C82EF2DB00BF4B
:109CB000C82E02DB0120BDE8F087B8F1020F09D100
:109CC000C4F3072000F0BCF9012803D100F0FFF92C
:109CD0000120F0E7E0B200F0B3F9012803D100F071
:109CE000F6F90120E7E700F0E7F947F0010000F09E
:109CF000A7F9B8B90BE000F07BF905F8010BB9F151
:109D0000000F02D000F05AF901E000F049F9B9F172
:109D10000000A9F1010101F0FF09ECD100F0D7F931
:109D20000020C8E700F0D3F90120C4E72DE9F0478F
:109D300082460C4617469846DDE9089541E0002624
:109D40000AE000F0B9F9504600F07AF900B905E0F0
:109D500000F0BDF9701CC6B2C82EF2DB00BFC82EE1
:109D600002DB0120BDE8F087022F09D1C4F30720F0
:109D700000F066F9012803D100F0A9F90120F1E70C
:109D8000E0B200F05DF9012803D100F0A0F9012054
:109D9000E8E711E019F8010B00F052F9012803D1AE
:109DA00000F095F90120DDE7681EC5B2641CA8F13A
:109DB0000100204000B901E0002DEBD100BF00F010
:109DC00086F9002DBBD10020CCE7000010B5254856
:109DD0000078002844D000202249087022480078EA
:109DE000012802D101F0FAFC01E001F051FC4FF42E
:109DF00000411E48FEF71BF8F0B91D480078022804
:109E000008D01B480078B8B91A480078A0B11A48A1
:109E1000408888B119480088401C80B217490880E2
:109E200041F27071884207DB0020144908804FF42A
:109E300000410E48FEF706F80D480078012808D0CA
:109E40000B48007850B90B48007810B10A48408898
:109E500020B94FF400410548FDF7F2FFFEF77AFE06
:109E600010BD000023000020760000200008014003
:109E70005E00002074000020FA0400205C00002036
:109E800010B50548007830B100200349087001F092
:109E900005F9FEF7E1FD10BD2200002010B52248B3
:109EA000007800283FD000201F4908701F48007824
:109EB00058B11F480078401CC0B21D4908700A28DC
:109EC00003DB00200870194908701A48007858B15F
:109ED00019480078401CC0B217490870022803DBFB
:109EE000002008701349087000F0F4FF00F06CF9CE
:109EF0001048007840B11148007828B10F48007828
:109F0000401E0E49087002E000200A4908700C4803
:109F1000007818B100200A49087004E00848007869
:109F2000401C0749087010BD240000205E0000207E
:109F30005F00002030000020600000203200002080
:109F40006E0000200148408870470000680400202F
:109F500002480088C0F30B00704700002A00002070
:109F600008B501210C20FEF793F803208DF80200BC
:109F700010208DF803004FF48C70ADF80000694696
:109F80000548FDF773FE4FF44060ADF800006946E8
:109F90000248FDF76BFE08BD00080140000C0140BF
:109FA00010B5002001F076FA012001F085FA0120B9
:109FB00001F070FA002001F06DFA10BD10B500201C
:109FC00001F068FA002001F077FA012001F062FA4E
:109FD000002001F05FFA012001F06EFA10BD10B50B
:109FE000012001F069FA012001F054FA10BD0000CF
:109FF00070B5012529031148FDF724FF00BF00209B
:10A0000001F048FA6006040E0A20FFF79FF80120CD
:10A0100001F040FA4FF480510848FDF7FBFE08B10B
:10A0200044F001046806050E002DE8D1002001F07F
:10A0300031FA0A20FFF78AF8204670BD0008014077
:10A0400070B50546802400BF002001F023FA05EA20
:10A05000040001F031FA0A20FFF778F8012001F03E
:10A0600019FA0A20FFF772F86410002CECD10020D6
:10A0700001F010FA4FF480510E48FDF7E3FE0A207C
:10A08000FFF764F8012001F005FA0A20FFF75EF8F7
:10A090004FF480510748FDF7BDFE0646002001F051
:10A0A000F9F90A20FFF752F80EB1012070BD002027
:10A0B000FCE700000008014010B5012001F0FCF9A8
:10A0C000012001F0E7F9002001F0F6F910BD10B50C
:10A0D000002001F0DFF9002001F0EEF9012001F08D
:10A0E000D9F9012001F0E8F910BD704710B52048FA
:10A0F000007803280ED11F48007B18B100201D49AD
:10A10000087302E001201B49087301F02BFDFFF7E3
:10A11000FFFC2BE016480078042811D11548407B3D
:10A12000002805DD1348407B401E1249487302E0B9
:10A1300014201049487301F015FDFFF743FB15E0AB
:10A140000B480078052811D10A48C0893C2805DB56
:10A150000848C0893C380749C88103E04FF496702D
:10A160000449C88101F0FEFCFFF758F810BD00005B
:10A1700076000020FA04002010B510480078E0B9FD
:10A180000F48C07A012818D10E480078012808D15C
:10A1900003200C490870052008490870FFF7B8FC37
:10A1A0000BE008480078032807D101200549087012
:10A1B000052002490870FFF771F810BD3300002038
:10A1C000FA0400207600002010B515480078012818
:10A1D00015D11448007830B103280BD0042806D0DC
:10A1E00005280AD100E009E000F0E0F806E0FFF7FA
:10A1F000C3FF03E000F058F800E000BF00BF0A48CA
:10A20000007858B109480078401CC0B2074908706E
:10A21000052803DB002008700349087010BD00000A
:10A2200031000020410000204500002046000020B1
:10A2300010B519480078012805D118490870022086
:10A240001749087021E01448007806280AD1072031
:10A2500011490870012000F00FFF01F00BF8FFF723
:10A2600029FB12E00C480078052805D104200A4992
:10A270000870FFF7A7FA08E007480078042804D11F
:10A28000052005490870FEF7C9FF06480078401C04
:10A290000449087010BD0000760000203000002046
:10A2A000320000204500002010B512480078F8B9AF
:10A2B0001148007801280BD110480078022807D1F6
:10A2C00005200D4908700B490870FEF7A7FF0FE045
:10A2D00009480078042803D007480078052807D1EA
:10A2E000012005490870052002490870FEF7D6FFD5
:10A2F00010BD000033000020760000205E0000202A
:10A3000010B52848007802281FD12748C07A30B1FC
:10A31000012808D002280AD0032810D10BE0012020
:10A320002149C8720BE002201F49C87207E00320D0
:10A330001D49C87203E000201B49C87200BF00BF5E
:10A3400001F010FCFFF7E8FA2AE01648007804282C
:10A3500011D11548407B142805DA1348407B401C76
:10A360001149487302E000200F49487301F0FAFBDD
:10A37000FFF728FA14E00B480078052810D10A48A6
:10A38000C089F02805DC0848C0893C300649C881EE
:10A3900002E000200449C88101F0E4FBFEF73EFF23
:10A3A00010BD000076000020FA04002010B50E4811
:10A3B0000078C0B90D480078012808D102200B4967
:10A3C0000870052008490870FFF7A6FA0BE0074857
:10A3D0000078022807D101200449087005200249AD
:10A3E0000870FEF75BFF10BD3300002076000020F0
:10A3F00010B51B480078062803D1012018490870C1
:10A400002DE018480078032808DB00201549087063
:10A41000062013490870FFF719FA20E01248007867
:10A4200040B911480078D0B910480078B8B1104848
:10A430004088A0B10E48407A88B9094800780128C0
:10A440000DD10B48807A18B100200949887202E0CA
:10A4500001200749887201F085FBFEF71FFF10BD40
:10A4600076000020450000205E00002074000020DF
:10A47000FA0400202DE9F84F80468946154615F864
:10A4800001AB15F8010B00900AF00707082F15D251
:10A49000DFE807F00406080A0C0E101280240EE014
:10A4A00001240CE002240AE0042408E0082406E069
:10A4B000102404E0202402E0402400E000BF00BF9C
:10A4C0004FF0000B2AE0B9F1400F00DD2DE02746E8
:10A4D00000261CE008EB0600602800DD19E0287863
:10A4E000384038B108EB0601C8B20122494601F0F4
:10A4F00069FB06E008EB0601C8B20022494601F0FC
:10A5000061FB7F100FB980276D1C701CC6B25645C9
:10A51000E0DB00BF09F1010000F0FF095846411CD3
:10A5200001F0FF0B00998842CDDB00BFBDE8F88F3A
:10A5300008B501210820FDF7ABFDFF20ADF80000B4
:10A5400003208DF8020010208DF8030069460948A9
:10A55000FDF78CFB01210846FDF79AFD0121064815
:10A56000FDF710FC1820ADF8000069460148FDF722
:10A570007DFB08BD000C0140000230002DE9F047D2
:10A5800006460F4690469946DDF820A034460CE07A
:10A590003D4606E052462946204601F013FB681C62
:10A5A000C5B24D45F6DD601CC4B24445F0DDBDE8E2
:10A5B000F0870000014606294DD2DFE801F04C0388
:10A5C00012212E3D0822254B1A700622244B1A70A8
:10A5D0000822244B1A705001234A121A234B1A6086
:10A5E0003AE010221D4B1A7008221D4B1A701022DF
:10A5F0001C4B1A7050011E4A121A1C4B1A602BE099
:10A600000822164B1A70164B1A70164B1A7050010E
:10A61000184A121A154B1A601EE00C220F4B1A70C2
:10A6200008220F4B1A700C220E4B1A705001124A5E
:10A63000121A0E4B1A600FE03022084B1A701022CB
:10A64000074B1A701822074B1A7090010B4A121A06
:10A65000064B1A6000E000BF00BF704700000020FA
:10A66000080000200900002034C600080400002073
:10A67000C4D200082CC9000844CE0008F4DC00084D
:10A6800008B501211C20FDF703FD4220ADF80000B4
:10A6900010208DF8030003208DF8020069461E4843
:10A6A000FDF7E4FA40F2FF30ADF8000010208DF81D
:10A6B000030003208DF8020069461848FDF7D6FA1A
:10A6C0004FF40050ADF8000010208DF80300032077
:10A6D0008DF8020069461248FDF7C8FA01210846C4
:10A6E000FDF7D6FC01210F48FDF74CFB4FF400406D
:10A6F000ADF8000003208DF8020010208DF8030053
:10A7000069460548FDF7B2FA1820ADF80000694621
:10A710000248FDF7ABFA08BD00080140000C0140FB
:10A7200000100140000230002DE9F04F04460D46B4
:10A730009046994600274FF0010B4D4507DD66B264
:10A74000444606F0FF086EB24D4606F0FF09A8EB3E
:10A75000040046B2A9EB05004FFA80FA29462046CC
:10A76000099A01F02FFA002E04DCA4EB080046B28F
:10A770004FF0FF3B56451CDD18E0002F06DD681C3E
:10A78000C5B2AAEB0600384447B202E007EB0A0064
:10A7900047B204EB0B00C4B2602C01DA402D00DBA1
:10A7A00006E029462046099A01F00CFA4445E4D116
:10A7B0001BE017E0002F07DD04EB0B00C4B2A6EB93
:10A7C0000A00384447B201E0B81947B2681CC5B264
:10A7D000602C01DA402D00DB06E029462046099A6C
:10A7E00001F0F0F94D45E5D100BFBDE8F08F000064
:10A7F0002DE9F04706460F4692463048006830493A
:10A8000009780AFB0109002551E099F8008000242D
:10A8100044E0072C16DC08F0800038B17A19D1B278
:10A820003219D0B2012201F0CDF906E07A19D1B285
:10A830003219D0B2002201F0C5F94FEA48604FEA60
:10A84000106826E009F10100814690F80080082494
:10A850001AE008F0800038B17A19D1B23219D0B2BA
:10A86000012201F0AFF906E07A19D1B23219D0B263
:10A87000002201F0A7F94FEA48604FEA1068602C07
:10A8800000DD05E0601CC4B20E4800788442E0DBC5
:10A8900000BF602C00DD05E0601CC4B209480078F0
:10A8A0008442B6DB00BF09F10109681CC5B2064845
:10A8B00000788542A9DBBDE8F08700000400002095
:10A8C00000000020080000200900002070B50546A7
:10A8D0000E46144615E00D4800782844602800DD37
:10A8E00012E00B4800783044402800DD0CE022786C
:10A8F00031462846FFF77CFF044800782844C5B25B
:10A90000641C20780028E6D100BF70BD080000203C
:10A91000090000202DE9F04DC84A002490B0914272
:10A9200005DA21F00043934201D805D120B110B0DF
:10A93000BDE8F04DFEF780B8B1F5801F1BDA53EA91
:10A94000000209D0002911DA0120FCF71BFE10B02B
:10A95000BDE8F04DFEF773B80220FCF713FEFEF7DA
:10A9600063F810B081F00041BDE8F08D6FF0350460
:10A97000362201F019FE04EB2152C1F31308B0494D
:10A98000A2F2FF33414401F4801282F07F6103EBB5
:10A99000225281F04051009241EA08010022A94B65
:10A9A00001F0E6FC044608F10200A74EC0F31300D4
:10A9B0000D467E44032867D2D6E90023204601F0E5
:10A9C00037FB1ED10098002802BFD6E9000110B065
:10A9D000BDE8F08D01F097FB07460C469B4A9C4B67
:10A9E00001F0BCFB06460D469A4A9B4B3846214671
:10A9F00001F0B4FB10B032462B46BDE8F04D01F03B
:10AA000003B94FF05532954B2046294601F0A6FB7D
:10AA10000022934B01F0A0FC06460F4622462B462F
:10AA20001046194601F09AFB32463B4601F096FB70
:10AA3000064600980F46F0B101F065FB80468A4655
:10AA4000824A834B01F08AFB32463B4601F084FC8C
:10AA500022462B4601F08CFC05460C467D4A7E4B77
:10AA60004046514601F07AFB10B02A462346BDE825
:10AA7000F04D01F07DBC0B4610B032462046294611
:10AA8000BDE8F04D01F074BC00224FF08043204639
:10AA900001F0BAF802460B462046294601F070F94B
:10AAA00006460F46009801F02EFBCDE90401324620
:10AAB0003B461046394601F051FB0C9069480C9A10
:10AAC0004044019009910B46104601F047FB824635
:10AAD000024665488B46C8F151080B4608F5D72851
:10AAE00003217844FDF74AFF52465B4601F036FBEE
:10AAF0000A905E480D9152465B4604217844FDF76A
:10AB00003DFF099B0C9A01F029FB844601980D9B9F
:10AB100040EA080860460A9A01F076F883460891F0
:10AB2000B8F1000F4EDD4FF0FF322046294601F00C
:10AB30003BFD22462B4601F011FB804600988A46D9
:10AB400060B3DDE90401414A414B01F007FB099183
:10AB500000905A4640465146089B01F055F832464F
:10AB60003B4601F0FBFA099B009A01F04DF8424682
:10AB7000534601F0F1FB22462B4601F0F9FB044657
:10AB80000D46DDE90401334A334B01F0E7FA10B01A
:10AB900022462B46BDE8F04D01F0EABB5A4640463E
:10ABA000089B01F031F832463B4601F0D7FA4246A5
:10ABB000534601F0D1FB10B022462B46BDE8F04DC4
:10ABC00001F0CABB009840B3DDE904011F4A204BE5
:10ABD00001F0C4FA80468A465A4620462946089B18
:10ABE00001F0C6FB32463B4601F0B8FA42465346F6
:10ABF00001F0BEFB22462B4601F0BAFB04460D468F
:10AC0000DDE90401134A144B01F0A8FA10B0224602
:10AC10002B46BDE8F04D01F0ABBB0B465A46204633
:10AC2000294601F0A5FB32463B4601F097FA10B0E9
:10AC300022462B46BDE8F04D01F08EBB0000F07FB0
:10AC4000645F09000000F03F6A470000763C7935F8
:10AC5000EF39EA3D0000E0FE422EE63F5555D53F74
:10AC60000000E03F86EBF9FF0246000000460000CE
:10AC70005E4800685E49B0FBF1F0C5B22846FEF7B9
:10AC80001BFAFDF78AF901214FF0C050FDF7F0F9EA
:10AC90000120FDF7CBF9FEF7D1FF54480068554974
:10ACA000B0FBF1F0401E85B229466320FDF7B6FCEB
:10ACB00000F02CFDFDF7F0FEFFF752F9FDF7E6F886
:10ACC000E220FDF70BF9E020FDF708F9A320FDF7DE
:10ACD00005F9A020FDF702F9C820FDF7FFF8AC2028
:10ACE000FDF7FCF8A620FDF7F9F8A420FDF7F6F82B
:10ACF0002C20FDF7F3F82E20FDF7F0F82F20FDF7BC
:10AD0000EDF82520FDF7EAF88120FDF7E7F80820A7
:10AD1000FDF7E4F8D520FDF7E1F80020FDF7DEF8B7
:10AD2000D220FDF7DBF80020FDF7D8F84020FDF732
:10AD3000D5F8B020FDF7D2F81020FDF7CFF80020AD
:10AD4000FDF7CCF84FF49670FEF7D4F9AF20FDF77D
:10AD5000C5F84FF400412848FDF772F8FEF760F996
:10AD600018B9FEF719FA00BFFEE724492448FCF79A
:10AD700098FB24A12248FCF756FB044634B1211D60
:10AD80002148FCF78EFB641E00202070FEF734FF84
:10AD900000201E4908701E49088000F0F7F800F0F6
:10ADA000D5F94FF400611B48FDF74AF84FF4806174
:10ADB0001848FDF745F810210F48FDF741F800202D
:10ADC00015490870154908701549488015490870DB
:10ADD0003C201549087000201449087005E0FFF771
:10ADE0004FF8FEF7F3FFFFF759F8F8E78C00002063
:10ADF00040420F00A086010000080140D6F0000884
:10AE0000EA04002056455200E004002076000020AD
:10AE100078000020000C01406F000020700000202E
:10AE2000FA04002054000020860000206D0000205D
:10AE30002DE9F04704460F4690469946B9F1000FB8
:10AE400007D0207B40F08001217384F80D900E25FF
:10AE500030E0207B04281AD10D254FEA4860020E0D
:10AE600029466D1C625400260EE037F816000212C7
:10AE70002846691CCDB2225417F816202846691CB2
:10AE8000CDB22254701CC6B24645EEDB12E0207BE8
:10AE9000052802D0207B10280CD10D25002607E0C4
:10AEA00017F816202846691CCDB22254701CC6B271
:10AEB0004645F5DB29462046FCF7C8FF82464FEAA7
:10AEC0002A206055611981F801A0A81CC0B2BDE814
:10AED000F087000010B51848007868B91748008856
:10AEE000401C80B215490880042823DB002008801C
:10AEF0000120114908701DE00F480078012808D191
:10AF00000F48007810B9FEF7C9F913E0FFF75CF9B4
:10AF100010E00A480088401C80B208490880782860
:10AF200008DB0020088004480078072802D00120B0
:10AF30000149087010BD0000760000207800002054
:10AF40003100002070B505460C4620780F281ADD28
:10AF50002078284410F8026C2078284410F8010C5E
:10AF600040EA06262078801E81B22846FCF76EFF54
:10AF7000B04205D1002020702846FDF7BBFE04E05A
:10AF80000020207001E00020207070BD38B5122430
:10AF900000BF402CFDDC1C4B01220021AE200094A0
:10AFA000FEF76EFE012802D11849087002E0002069
:10AFB00016490870A01E81B21348FCF747FF1249DA
:10AFC000098A88421AD0104B01224021AE200094F9
:10AFD000FEF756FE012802D10C49087002E000205D
:10AFE0000A490870A01E81B20748FCF72FFF0649E6
:10AFF000098A884202D0012000F03EF82246024928
:10B000000348FCF772FA38BDFA0400204F00002014
:10B010000C05002010B5FEF795FF044640F63C7085
:10B02000844203DD00201349087021E040F64850B7
:10B03000844203DD01200F49087019E040F68C209E
:10B04000844203DD02200B49087011E040F26C706D
:10B05000844203DD03200749087009E0B4F5AF7F9F
:10B0600003DD04200349087002E00520014908704F
:10B0700010BD00003900002010B50446002006492C
:10B080008872C87201200873002048734FF49670CC
:10B09000C88100F067FD10BDFA04002010B58021C2
:10B0A0000A48FCF7C4FE80B909480078401CC0B2C9
:10B0B00007490870022808DB00200870054800785E
:10B0C00018B104490448FFF73DFF10BD00080140D6
:10B0D0002700002028000020A003002010B504460F
:10B0E00000200A4908700A48047080210948FCF7CA
:10B0F000A9FE0020084908700878411C064A117012
:10B100000649095C064A118010BD00002700002096
:10B11000290000200008014028000020A003002092
:10B12000043801400748008807490860084600883D
:10B13000000408600348001D0088096808440249AB
:10B1400008607047182800407C00002070B5002679
:10B150000420FCF75BFC012832D001214FF0C050E5
:10B16000FCF786FF0120FCF761FFFCF746FC01209D
:10B17000FDF73CF800BF4120FDF71AF80028FAD08F
:10B180004FF48070FDF752F80120FDF749F8FDF704
:10B1900033F9FDF73BF901210846FDF70DF9FDF7FD
:10B1A0002BF9FDF753F847F6FF70FDF715F9FDF79A
:10B1B00023F9FDF755F801210420FCF735FC07E0E1
:10B1C000FDF724F901210846FDF7F6F8FDF714F91B
:10B1D000FFF7A8FF0C20FCF719FC06461020FCF72F
:10B1E00015FC40EA06461420FCF710FC0446182023
:10B1F000FCF70CFC054604B9F5B135B11248C0891D
:10B2000012490968891B441A03E010480068801B32
:10B21000241A002C03DA00200D49088001E00C49B3
:10B220000C800948C0890A490988884207DA06481B
:10B23000C0890749088002E000200549088000F025
:10B2400009F8002070BD0000FA0400207C000020F6
:10B250007200002008B503208DF8000000208DF852
:10B2600001008DF8020001208DF803006846FCF70C
:10B270009BFE08BD10B501214FF0C050FCF7F8FE51
:10B280000120FCF7D3FEFCF7B8FB00210120FDF7FD
:10B2900093F8FDF7B1F80020FCF7C2FF0020FCF79F
:10B2A000A5FF0020FCF7C2FE00214FF0C050FCF7C4
:10B2B000DFFE10BD10B5FFF7ADFE60480078062830
:10B2C00079D2DFE800F0034E5C6A79875C48007849
:10B2D000002845D15B48007818B900205A49087009
:10B2E0003EE05A48006800283AD0584800680528CF
:10B2F0002FD956480068B0F5967F2AD25148007879
:10B30000514908700846007818B3084600780628A6
:10B3100013D2DFE800F0120C0903060FFEF788FFD6
:10B320000CE0FEF7E3FE09E0FFF762F806E0FEF747
:10B33000DCFE03E0FEF7E4FF00E000BF00BF4FF4D7
:10B3400000414348FCF77CFD002042490880424907
:10B3500008800020414908703C4908604049087055
:10B3600047E037480078012808D13648007801289E
:10B3700004D136480068401C3449086039E0304840
:10B380000078022808D12F480078022804D12F48DD
:10B390000068401C2D4908602BE0294800780328EC
:10B3A00008D128480078032804D128480068401CA8
:10B3B000264908601DE01BE021480078042808D1D8
:10B3C00020480078042804D120480068401C1F4908
:10B3D00008600EE01A480078052808D1194800785E
:10B3E000052804D119480068401C1849086000E08D
:10B3F00000BF00BF12480078124908700F4800785B
:10B400000F49087011480068B0F5967F15D90F48AC
:10B410000068401E0D490860012010490870074867
:10B420000078104908704FF400410948FCF708FD06
:10B430000020084908800849088010BD3900002014
:10B440003700002038000020400000203C00002091
:10B45000000801405C00002078000020310000203E
:10B4600036000020410000200648007848B1002046
:10B47000044908700448C089044908803C200449F4
:10B480000880704780000020FA040020720000202D
:10B490008200002010B504462CB14FF4006105482D
:10B4A000FCF7D0FC04E04FF400610248FCF7C8FC54
:10B4B00010BD00000008014010B504462CB14FF447
:10B4C00080510548FCF7BEFC04E04FF4805102486F
:10B4D000FCF7B6FC10BD00000008014010B52D4877
:10B4E000008800284ED12C48C07A01281FD12A4854
:10B4F000007B70B14FF480612848FCF798FCB0B92C
:10B500000320274908704FF480612448FCF79AFC17
:10B510000DE04FF480612148FCF789FC38B103202D
:10B520001F4908704FF480611C48FCF789FC1C48D7
:10B53000007838BB4FF400611848FCF778FC80B9FC
:10B5400018480078184908701848007848B9184811
:10B55000007830B91048407B144908700120144924
:10B5600008701248007850B911480078012806D1B7
:10B57000C1020A48FCF766FC00200D490870012052
:10B580000C49087001200C49087000200B49087014
:10B5900010BD000072000020FA040020000C0140E1
:10B5A00084000020860000206C0000208500002020
:10B5B00075000020800000206F0000207000002037
:10B5C00010B52A48C07A012839D1294800880028B6
:10B5D00044D12648007B70B14FF480612548FCF7C8
:10B5E00026FCB0B10320244908704FF48061214843
:10B5F000FCF726FC0DE04FF480611E48FCF717FCB9
:10B6000038B903201C4908704FF480611948FCF7D1
:10B6100019FC1948007808BB4FF400611548FCF785
:10B6200006FC18B915480078154908704FF40061F8
:10B630001048FCF707FC0120124908700EE04FF497
:10B6400080610C48FCF7F3FB18B90C4800780C49F2
:10B6500008704FF480610748FCF7F4FB00200A49AA
:10B66000087001200949087010BD0000FA0400208C
:10B6700072000020000C01408400002086000020A1
:10B680006C000020800000206F000020700000206F
:10B6900010B51648007820B94FF400611448FCF743
:10B6A000CFFBFFF7E1FE4FF480611148FCF7BFFBD1
:10B6B00058B11048C07A012807D03C200E490880B4
:10B6C0004FF480610A48FCF7BBFB4FF480710B48D4
:10B6D000FCF7B6FB08210948FCF7B2FB002008493B
:10B6E0000870084908700849087010BD84000020DF
:10B6F000000C0140FA0400208200002000080140F4
:10B700006F000020700000206D00002000B587B0A1
:10B71000012144F20400FCF7BBFC03208DF81A0061
:10B7200010208DF81B008020ADF8180006A92948CC
:10B73000FCF79CFA03208DF81A0018208DF81B00E6
:10B740004FF40070ADF8180006A92248FCF78EFAF5
:10B7500048208DF81B004FF48060ADF8180006A952
:10B760001C48FCF783FA4FF4964002900020ADF895
:10B770000C00ADF80E00ADF81000ADF814000C2070
:10B78000ADF8120002A91448FDF78AF8012240F230
:10B7900025511148FDF75EF8012240F226610E485E
:10B7A000FDF758F801210C48FDF73BF825208DF8EE
:10B7B000040000208DF805008DF8060001208DF8AA
:10B7C000070001A8FCF7F0FB80210248FCF738FBDA
:10B7D00007B000BD000801400038014070B5AB481B
:10B7E000407A022803D0A948407A032803D10520D3
:10B7F000A749087002E03C20A5490870A5480078D8
:10B8000010B9A5480078B0B9A2480078012802D143
:10B81000A248007878B19D48407A01280BD0A04812
:10B8200000884FF6FF71884205D09D48008810B10E
:10B830009648408858B9FFF72BFF4FF4806199482C
:10B84000FCF7FEFA10219848FCF7FAFA1DE18F4840
:10B85000807A10B99548008820B110219248FCF7F1
:10B86000F1FA03E010219048FCF7EAFA8748007AE1
:10B8700010B18648448801E0844884888348C07AAF
:10B8800003283ED18148807920448549098888422F
:10B8900002DAFFF723FE05E081480088A04201DAC2
:10B8A000FFF7F6FE08218048FCF7CAFA774880794E
:10B8B00004EB40007A490988884212DA4FF40061AB
:10B8C0007848FCF7B4FA60B10120794908707948EA
:10B8D00000780028BAD14FF480717348FCF7B2FAAF
:10B8E000D3E06A48807920446D4909888842ADDDFB
:10B8F0004FF480716C48FCF7A3FA00206C49087083
:10B90000C3E06248C07A02283DD160488079201A9D
:10B9100063490988884202DDFFF752FE05E060486E
:10B920000088A04201DDFFF7B3FE4FF480715E484E
:10B93000FCF786FA55488079A4EB400058490988FD
:10B94000884211DD4FF480615648FCF770FA58B117
:10B95000012057490870574800780028C0D10821B5
:10B960005148FCF76FFA90E048488079201A4C491A
:10B970000988884206DA08214B48FCF761FA002062
:10B980004B49087081E041488079201A4449098870
:10B99000884230DD4848007810B1FFF779FE74E046
:10B9A000FFF70EFE4FF480713F48FCF749FA374825
:10B9B000C07A012805D1C1023A48FCF738FA054699
:10B9C00005E04FF480613748FCF731FA05462F480F
:10B9D0008079A4EB400032490988884255DDB5B32F
:10B9E0000120334908703348007880BB08212E4875
:10B9F000FCF728FA49E0254880792044284909883D
:10BA0000884225DA2D48007810B1FFF741FE3CE06E
:10BA1000FFF764FD08212448FCF712FA1B488079DF
:10BA200004EB40001E49098888422EDA4FF4006179
:10BA30001C48FCF7FCF950B101201D4908701D4855
:10BA4000007820B94FF480711748FCF7FBF91CE02F
:10BA50001948007818B112480088A04206DB174840
:10BA6000007830B10E480088A04202DDFFF710FEDA
:10BA70000BE008210C48FCF7E3F94FF480710A4809
:10BA8000FCF7DEF900200A49087070BDFA040020B6
:10BA9000860000205E000020550000207400002079
:10BAA00064000020000C01400008014082000020DA
:10BAB0006D0000206C0000206F000020700000204E
:10BAC0002DE9F84305460E4617469846DDE9084934
:10BAD00033463A46314628460094FEF725FE434653
:10BAE0002A46314628460094FEF71EFE43463A4653
:10BAF000414628460094FEF717FE43463A46314633
:10BB000038460094FEF710FE43463A463146284632
:10BB1000CDF80090FEF732FDBDE8F88370B5002542
:10BB200000240F4E00BF17E0B02141EAE400FCF70B
:10BB3000D5F91020FCF7D2F90020FCF7CFF9002549
:10BB400005E016F8010BFCF7F7F9681CC5B2602D8B
:10BB5000F7DB04F10800C4B2402CE5DD70BD000045
:10BB6000A00000201CB51224A01E81B21348FCF7CF
:10BB70006DF9124908820846102301220021CDE9FF
:10BB80000004AE20FEF7D2F8012802D10C4908705B
:10BB900002E000200A4908700848102301224021D1
:10BBA000CDE90004AE20FEF7C1F8012802D1044916
:10BBB000087002E00020024908701CBDFA04002051
:10BBC0004F00002070B5034601F007060125B5407F
:10BBD000ECB2CD1005EB45050A4E06EB4515E85CC9
:10BBE000012A01D1204305E00AB9A04302E0022A5C
:10BBF00000D16040CD1005EB4505024E06EB451522
:10BC0000E85470BDA000002010B591EA030F48BFB2
:10BC100083F0004300F1B483841A71EB030C05D266
:10BC2000121943EB0C03001B61EB0C01DFF824E15C
:10BC30004FEA1154A4EB135C1EEA430F18BF9EEAAF
:10BC4000445F73D023EA0E03DCF1200E21EA045195
:10BC500043F4801332D322FA0CFE10EB0E0023FAC9
:10BC60000CFE41EB0E01CCF1200E03FA0EFE10EBA0
:10BC70000E0051F10001B1F5801FCCF1200E32D23F
:10BC800001EB045112FA0EF2BDE8104058BF7047A4
:10BC9000401C38BF5FEA420218BF7047002814BF3B
:10BCA00020F0010041F100014FEA410313F5001FAC
:10BCB00038BF7047A1F1C04100F048BB012A43EBF7
:10BCC0000302ACF1200CDCF11F0E32BF4FF0000E6E
:10BCD00023FA0CF310EB030041EB0451B4EB115FBA
:10BCE000D0D0A1EB045101F5801149085FEA300082
:10BCF00001EB04510ED350F1000038BF12FA0EFED2
:10BD000008D1BDE81040C9E7401C38BF5FEA4202D5
:10BD1000CAD1C3E7BDE810404FEA410313F5001F45
:10BD200038BF7047A1F1C04100F010BB9EEA445FEC
:10BD300008D011EA5E0FBDE8104004BF01F00041D9
:10BD400000207047BDE8104070B500F0B1FA00BFA8
:10BD500064FBBE3E0000E0FF02494FF0000000F02F
:10BD6000F1BB00BF0000F87F491058BFC1F140414E
:10BD70005B1058BFC3F140438B42EFF30080704724
:10BD80002DE9C04130B4DFF8A0C23CEA111418BF5D
:10BD90003CEA131400F0EC8081EA03051CEA11145C
:10BDA00044EAD57418BF1CEA131500F0C780A4EB51
:10BDB00005044FF0004545EAC12145EAC32341EAA5
:10BDC000505143EA525304F17F74994204F5003410
:10BDD0004FEAC0204FEAC22208BF904200F09C8088
:10BDE0004FEA13650FF24016765D4FEA134506FBE6
:10BDF00005F7C7F1807706FB07F74FEAD737A7FBB0
:10BE000003687642C8F58038A7FB06CE38BFA8F194
:10BE1000010807FB08E64FF0000EA6FB028CE6FBCC
:10BE200003CEDCF1000CCEF1004E38BFAEF1010EB6
:10BE3000A6FB0C584FF000074FF00005E6FB0E87FD
:10BE4000A1FB08C6A0FB07CE16EB0E0645F10005C8
:10BE5000E1FB076515F1E04E7EBFA4F580345FEA93
:10BE600046066D4116F1800745F100054FEA172798
:10BE70004FEA066647EA0567A6F1DE46B6F1805F3F
:10BE80004FEA15251FD9384624F0010C05EBC47183
:10BE9000BCF1FE6F01EB0C1102D8F0BCBDE80081D3
:10BEA00024425CBF01F5801E9EEAC47F02D4F0BC30
:10BEB000BDE80081244238D4F0BCA1F1C041BDE806
:10BEC000004100F043BA4FEAD22242EA43524FEA1D
:10BED000D323A7FB02864FEAD02040EA415007FB5C
:10BEE00003661EEA0E0F4FEAD12105FB026658BF1A
:10BEF000A6EB0056B6EB00564FEA520E4EEAC37E52
:10BF000018EB0E0E56EB530EBDD518EB02085E4132
:10BF10007F1C55F10005B6E74FF480154FF0000780
:10BF20004FF000064FF00008ADE7F0BC4FF0000006
:10BF300001F1C04101F00041BDE8008111EA0C1F90
:10BF40000CEA131500D00CE013EA0C1F00F025805A
:10BF50004FF00000F0BC81EA030101F00041BDE8B0
:10BF60000081F0BCBDE8004181EA030100F0EEB9B8
:10BF7000F0BCBDE8004170B500F09AF9097EFC3EC6
:10BF800000F007B881EA03014FF0000001F0004122
:10BF9000704781EA030100F0D9B9F0BCBDE8004167
:10BFA0004FF0000021497047FFFDFBF9F7F5F4F26F
:10BFB000F0EEEDEBE9E8E6E4E3E1E0DEDDDBDAD844
:10BFC000D7D5D4D3D1D0CFCDCCCBCAC8C7C6C5C4A2
:10BFD000C2C1C0BFBEBDBCBBBAB9B8B7B6B5B4B3B9
:10BFE000B2B1B0AFAEADACABAAA9A8A8A7A6A5A4A4
:10BFF000A3A3A2A1A09F9F9E9D9C9C9B9A99999868
:10C000009797969595949393929191908F8F8E8E0A
:10C010008D8C8C8B8B8A8989888887878685858497
:10C0200084838382828181800000FF070000F87F83
:10C0300051EA030C17D41CF5801F58BFBCF5801FB4
:10C0400000F10680994218BF704708BF90427047C0
:10C0500007D711F5801F58BF13F5801F19D49942D7
:10C060007047894270471CF5801F08D5BCF5801FBA
:10C07000F7D58B4218BF704708BF824270474FF414
:10C08000001C1CEB410F38BF1CEB430F01D28B424D
:10C09000704770B500F00CF9922449004FF0005140
:10C0A0004FF08053FFF760BE4FEA41034FEA53530E
:10C0B000A3F58063D3F11E03C8BFD3F1210C0CDDBF
:10C0C0004FF0004242EAC12242EA505232FA03FCE7
:10C0D0008CEAE17CACEBE1707047102BC4BF002010
:10C0E000704703F5787CBCF1FF3F04D06FF000424D
:10C0F00082EA2100704770B500F0DAF84992248096
:10C1000000207047F2E710F0004248BF4042B0FA0A
:10C1100080F310FA03F10AD0C3F11D0303F5806325
:10C120004FEA415002EB035202EBD12170474FF02E
:10C1300000007047B0FA80F310FA03F10AD0C3F19F
:10C140001D0303F580634FEA41504FEA035202EBAF
:10C15000D12170474FF0000070470000DFF848C160
:10C1600070B51CEA111E1EBF1CEA13159EEA0C0FC7
:10C1700095EA0C0F00F06F8081EA030423EA4C1368
:10C180004EEAD47E21EA4C1141F4801143F480132D
:10C19000AE44A1FB024CA0FB0365AEF17F7E3619D5
:10C1A00055EB0C05A1FB034C4CF10003A0FB021C5A
:10C1B00016EB0C06654153F10003094218BF46F027
:10C1C000010613F4007F0BD14FEA03314FEA05302B
:10C1D000340341EA155140EA16506FF003020AE0B9
:10C1E0004FEAC3214FEAC520F40241EA555140EA23
:10C1F00056506FF0020202EB2E4201EB025585EA27
:10C20000CE710AD05FEA440C18BF24F0004450F10C
:10C21000000041F1000120EAD47040F2FE7C62454A
:10C2200000D270BDA84214BF4FF080444FF040448C
:10C23000002E08BF0024BEF1806FA8BFA1F1C0414D
:10C24000BDE8704080F282804FF0000001F1C041F3
:10C2500001F0004170479EEA0C0F0CEA131518BF5D
:10C2600095EA0C0F06D04FF0000081EA030E0EF0A5
:10C27000004170BD00F01CF88900013E00F007B8D5
:10C2800000F009B84FEA430C5FEA5C5C08D081EA31
:10C29000030100F05BB84FEA410C5FEA5C5CF6D149
:10C2A0004FF00000014970470000FF070000F87FD1
:10C2B0000EF1020E2EF0030E5EF8046B364205D42A
:10C2C000012A43EB030515F5001F12D8012841EBA5
:10C2D000010C1CF5001F0CD80ED14FEAD17C15F5CE
:10C2E000001F0CEB4C0C0CF1020C08BF4CEBD37C88
:10C2F00004E04FF0080C01E04FEAD37C0CEB4C0556
:10C3000026FA05F606F00706B6F1040C06D20EEB87
:10C31000860CBDE870404CF0010C6047DFE80CF083
:10C32000090B02024FF000414FF00000A1F500217F
:10C3300070BD19461046012851EB010418BFD4F511
:10C34000001484BF002001F0004170BD0808A0F572
:10C3500000114FEA3101704791EA030F10B581F0E7
:10C3600000413FF559AC83F0004300F009B80000EC
:10C3700010B591EA030F48BF83F000433FF54CAC82
:10C38000841A71EB030C07D212198CF0004C43EBAA
:10C390000C03001B61EB0C01DFF8A4E14FEA115420
:10C3A000A4EB135C1EEA430F18BF9EEA445F00F043
:10C3B000B08023EA6E03524221EA0451C3EB6E03BC
:10C3C00038BF5B1EDCF1200E25D322FA0CFE10EBE9
:10C3D0000E0043FA0CFE41EB0E01CCF1200E03FAE5
:10C3E0000EFE10EB0E0051F10001CCF1200E29D40D
:10C3F00012FA0EF201EB0451BDE8104058BF70472D
:10C40000401C1CBFB2F1004F704700280CBF491CF4
:10C4100020F00100704712EB020E43EB030218BF3D
:10C420004FF0010E4EEA4202ACF1200CDCF11E0E80
:10C4300054D943FA0CFE10EB0E0051F1FF31CCF150
:10C440001E0ED5D50EF1010E12FA0EFE404141EB43
:10C45000010101EB445C5FEA5C5C10D910EBDE701B
:10C4600001EB045138BFBEF1004FBDE8104018BFCA
:10C47000704700280CBF491C20F00100704730D2E3
:10C480004FEAD42C11F5001124F400641BD0B1FA4A
:10C4900081F20B3AA41AA41ED2F12003914030FA83
:10C4A00003F31943904001EBCC71002C01EB0451D4
:10C4B000BDE81040A8BF704701F1C0414FF0000037
:10C4C00001F000417047B0FA80F310FA03F100D197
:10C4D00010BDE41A173C4805C90AE4E701EB045112
:10C4E00010BD491001EB0451BDE810404FEA300087
:10C4F00002E04FF0000170474A0008BF0042F8D048
:10C50000B2F5001F28BF704701F000414FF0000056
:10C5100070479EEA445F07D011EA5E0FBDE8104005
:10C5200004BF002100207047BDE8104070B5FFF740
:10C53000BFFE00BF40DFF63E83F00041104670476B
:10C540000000E0FF0CF00F03092B08BF082000F0EB
:10C5500059800A2B0BD0082B18BF704708BF1CF05E
:10C56000400F0AD04FF000004FF0000170471CF060
:10C57000400F18BF4FF0004070471CF0100F08D05C
:10C5800020F0704300F07F4242EAD3014FEA43704B
:10C59000704700F0604021F07F4242EA000201F063
:10C5A0007F4040EA727070474FF0FF0C4CF4E06C33
:10C5B0001CEA11531CBF9CEA030C9445C2BFDA422B
:10C5C00001EB02517047002B0DD0BCF1000F0FD0D2
:10C5D000002A01F00041A4BF41F0E04141F07F6139
:10C5E0004FF00000704701F000414FF0000070472D
:10C5F00050EA01334FF09B0C18BF4CF0806C7FF475
:10C60000ABAB70471CF4801F11D01CF4E02F03D09B
:10C610006FEACC31490070474FF04050EFF3008291
:10C6200022F0704242EA000282F3008870474FF025
:10C6300000007047000000000000000020202020C3
:10C640002000200048484800000000005050F850EA
:10C65000F85050002078A07028F02000C0C81020AA
:10C66000409818006090A040A890680060204000AA
:10C67000000000001020404040201000402010101A
:10C6800010204000005020F820500000002020F82A
:10C69000202000000000000000602040000000F8A2
:10C6A0000000000000000000006060000008102092
:10C6B00040800000708898A8C88870002060202002
:10C6C00020207000708808304080F80070880830A2
:10C6D0000888700010305090F8101000F880F008B2
:10C6E00008887000304080F088887000F8081020BA
:10C6F0004040400070888870888870007088887812
:10C700000810600000606000606000000000606071
:10C710000060204010204080402010000000F80001
:10C72000F800000080402010204080007088081031
:10C730002000200070880868A8A87000708888F819
:10C7400088888800F08888F08888F0007088808069
:10C7500080887000E09088888890E000F88080F001
:10C760008080F800F88080F0808080007088808071
:10C7700098887800888888F8888888007020202029
:10C780002020700038101010109060008890A0C019
:10C79000A0908800808080808080F80088D8A8A839
:10C7A000888888008888C8A89888880070888888C1
:10C7B00088887000F08888F0808080007088888881
:10C7C000A8906800F08888F0A09088007088807039
:10C7D00008887000F8202020202020008888888881
:10C7E000888870008888888888502000888888A871
:10C7F000A8A85000888850205088880088888850D1
:10C8000020202000F80810204080F80070404040B0
:10C810004040700000804020100800007010101090
:10C820001010700020508800000000000000000080
:10C83000000000F840201000000000000000700818
:10C84000788878008080B0C88888F0000000708008
:10C8500080887000080868988888780000007088D0
:10C86000F8807000304840E0404040000000788888
:10C87000887808708080B0C8888888002000602090
:10C88000202070001000301010109060808090A068
:10C89000C0A0900060202020202070000000D0A8C0
:10C8A000888888000000B0C88888880000007088E8
:10C8B000888870000000F08888F080800000788808
:10C8C000887808080000B0C8808080000000788068
:10C8D0007008F0004040E040404830000000888888
:10C8E00088986800000088888850200000008888A8
:10C8F000A8A85000000088502050880000008888B8
:10C90000887808700000F8102040F80010202040BF
:10C910002020100020202020202020004020201057
:10C92000202040006890000000000000000000008F
:10C9300000000000183C3C1818001800666624002F
:10C94000000000006C6CFE6CFE6C6C00183E603CDD
:10C95000067C180000C6CC183066C600386C3876E5
:10C96000DCCC760018183000000000000C183030C5
:10C9700030180C0030180C0C0C18300000663CFF0E
:10C980003C6600000018187E181800000000000027
:10C99000001818300000007E0000000000000000B9
:10C9A00000181800060C183060C08000386CC6C62D
:10C9B000C66C38001838181818187E007CC6061C7B
:10C9C0003066FE007CC6063C06C67C001C3C6CCC77
:10C9D000FE0C1E00FEC0C0FC06C67C003860C0FC19
:10C9E000C6C67C00FEC60C18303030007CC6C67C43
:10C9F000C6C67C007CC6C67E060C780000181800EF
:10CA0000001818000018180000181830060C18300C
:10CA1000180C060000007E00007E00006030180C3C
:10CA2000183060007CC60C18180018007CC6DEDECA
:10CA3000DEC07800386CC6FEC6C6C600FC66667CE2
:10CA40006666FC003C66C0C0C0663C00F86C66666A
:10CA5000666CF800FE6268786862FE00FE626878C4
:10CA60006860F0003C66C0C0CE663A00C6C6C6FE2E
:10CA7000C6C6C6003C18181818183C001E0C0C0C32
:10CA8000CCCC7800E6666C786C66E600F06060609E
:10CA90006266FE00C6EEFEFED6C6C600C6E6F6DE3E
:10CAA000CEC6C6007CC6C6C6C6C67C00FC66667C12
:10CAB0006060F0007CC6C6C6C6CE7C0EFC66667C96
:10CAC0006C66E6003C6630180C663C007E7E5A18A8
:10CAD00018183C00C6C6C6C6C6C67C00C6C6C6C6B2
:10CAE000C66C3800C6C6C6D6D6FE6C00C6C66C3844
:10CAF0006CC6C6006666663C18183C00FEC68C18FC
:10CB00003266FE003C30303030303C00C0603018BF
:10CB10000C0602003C0C0C0C0C0C3C0010386CC6D3
:10CB20000000000000000000000000FF30180C00B2
:10CB3000000000000000780C7CCC7600E0607C6691
:10CB40006666DC0000007CC6C0C67C001C0C7CCC89
:10CB5000CCCC760000007CC6FEC07C003C6660F851
:10CB60006060F000000076CCCC7C0CF8E0606C7665
:10CB70006666E6001800381818183C00060006061D
:10CB80000666663CE060666C786CE600381818183B
:10CB900018183C000000ECFED6D6D6000000DC667B
:10CBA0006666660000007CC6C6C67C000000DC66C7
:10CBB000667C60F0000076CCCC7C0C1E0000DC763D
:10CBC0006060F00000007EC07C06FC003030FC306D
:10CBD00030361C000000CCCCCCCC76000000C6C6A1
:10CBE000C66C38000000C6D6D6FE6C000000C66CCD
:10CBF000386CC6000000C6C6C67E06FC00007E4C2F
:10CC000018327E000E18187018180E001818181810
:10CC1000181818007018180E1818700076DC00002C
:10CC2000000000000C100000000000006010000078
:10CC3000000000007C82000000000000C600000030
:10CC400000000000728C0000000000000000381896
:10CC500018183C00386C6C7866666CC018003C662E
:10CC60007E6666003000780C7CCC76001E78989E3C
:10CC7000F8989E007C6666F666667C00F0607C66CE
:10CC8000667C60F00000CC327EB0EC006830580C5E
:10CC90007EC67C0070303C363C3078003A6CCED694
:10CCA000E66CB80000027CCED6E67C8000007CC634
:10CCB000FEC6C6000000FE607C60FE0000003C185E
:10CCC00018183C0000007CC6C6C67C000000C6C622
:10CCD000C6C67C000000E6F6DECEC60018001818B6
:10CCE0003C3C18003000303060C67C000C10000066
:10CCF0000000000060100000000000003844000048
:10CD000000000000C600000000000000728C00005F
:10CD10000000000000000000000000100000000003
:10CD20000000000000107CD0D0D67C101C30307881
:10CD300030325C00000044382838440044287C101D
:10CD40007C10100030303000303030003840304837
:10CD500030087000C6000000000000007E425A5EED
:10CD60005A427E0038043C443800000000366CD83B
:10CD70006C3600000000007C040400000000007C11
:10CD8000000000007C4454444C547C007C000000B3
:10CD900000000000304830000000000010107C103F
:10CDA00010007C0060902040F0000000E010601057
:10CDB000E00000000E182000000000000000666681
:10CDC00066667CC07ED4D47414143E000000001843
:10CDD0001800000040C04040E00000003C6666666D
:10CDE0003C00000000D86C366CD80000848890A409
:10CDF0004C941E04848890AC5284081EC0204024A9
:10CE0000CC141E0400663C183C6600000018007E2E
:10CE100000180000103070FC70301000203038FC1A
:10CE200038302000002070F820200000002020F87A
:10CE30007020000000082868F86020000606060C34
:10CE40008CD87830000000000000000000000000D6
:10CE50000030787878303000303000000066666648
:10CE60002400000000000000006C6CFE6C6C6CFE86
:10CE70006C6C000030307CC0C0780C0CF830300096
:10CE8000000000C4CC183060CC8C00000070D8D8F2
:10CE900070FADECCDC76000000303030600000003C
:10CEA00000000000000C183060606030180C0000BA
:10CEB000006030180C0C0C18306000000000006698
:10CEC0003CFF3C660000000000000018187E1818A7
:10CED0000000000000000000000000003838600082
:10CEE0000000000000FE0000000000000000000044
:10CEF0000000000038380000000002060C18306006
:10CF0000C0800000007CC6CEDED6F6E6C67C0000FF
:10CF1000001030F03030303030FC00000078CCCCE5
:10CF20000C183060CCFC00000078CC0C0C380C0CD9
:10CF3000CC780000000C1C3C6CCCFE0C0C1E0000DD
:10CF400000FCC0C0C0F80C0CCC780000003860C0F9
:10CF5000C0F8CCCCCC78000000FEC6C6060C183059
:10CF6000303000000078CCCCEC78DCCCCC78000001
:10CF70000078CCCCCC7C1818307000000000003851
:10CF80003800003838000000000000383800003851
:10CF900038183000000C183060C06030180C0000E9
:10CFA000000000007E007E000000000000603018DD
:10CFB0000C060C18306000000078CC0C18303000E3
:10CFC00030300000007CC6C6DEDEDEC0C07C000063
:10CFD000003078CCCCCCFCCCCCCC000000FC66661D
:10CFE000667C666666FC0000003C66C6C0C0C0C6C3
:10CFF000663C000000F86C66666666666CF80000C9
:10D0000000FE6260647C646062FE000000FE666296
:10D01000647C646060F00000003C66C6C0C0CEC6A0
:10D02000663E000000CCCCCCCCFCCCCCCCCC000000
:10D03000007830303030303030780000001E0C0C7A
:10D040000C0CCCCCCC78000000E6666C6C786C6C78
:10D0500066E6000000F060606060626666FE0000E8
:10D0600000C6EEFEFED6C6C6C6C6000000C6C6E6B0
:10D07000F6FEDECEC6C6000000386CC6C6C6C6C602
:10D080006C38000000FC6666667C606060F0000042
:10D0900000386CC6C6C6CEDE7C0C1E0000FC666680
:10D0A000667C6C6666E600000078CCCCC07018CC5C
:10D0B000CC78000000FCB4303030303030780000E4
:10D0C00000CCCCCCCCCCCCCCCC78000000CCCCCC24
:10D0D000CCCCCCCC7830000000C6C6C6C6D6D66C48
:10D0E0006C6C000000CCCCCC783078CCCCCC000080
:10D0F00000CCCCCCCC7830303078000000FECE981C
:10D1000018306062C6FE0000003C303030303030F5
:10D11000303C0000000080C06030180C06020000A7
:10D12000003C0C0C0C0C0C0C0C3C000010386CC6B9
:10D1300000000000000000000000000000000000EF
:10D140000000FF0030301800000000000000000068
:10D1500000000000780C7CCCCC76000000E0606021
:10D160007C66666666DC00000000000078CCC0C00B
:10D17000CC780000001C0C0C7CCCCCCCCC76000015
:10D180000000000078CCFCC0CC78000000386C6057
:10D1900060F8606060F000000000000076CCCCCC4D
:10D1A0007C0CCC7800E060606C76666666E6000019
:10D1B0000018180078181818187E0000000C0C00D1
:10D1C0003C0C0C0C0CCCCC7800E06060666C786C8D
:10D1D00066E600000078181818181818187E000065
:10D1E00000000000FCD6D6D6D6C600000000000025
:10D1F000F8CCCCCCCCCC00000000000078CCCCCC5F
:10D20000CC78000000000000DC666666667C60F09A
:10D210000000000076CCCCCCCC7C0C1E00000000C2
:10D22000EC6E766060F000000000000078CC6018C2
:10D23000CC78000000002060FC6060606C3800006A
:10D2400000000000CCCCCCCCCC760000000000006C
:10D25000CCCCCCCC7830000000000000C6C6D6D6BE
:10D260006C6C000000000000C66C38386CC6000012
:10D2700000000000666666663C0C18F000000000C6
:10D28000FC8C1860C4FC0000001C303060C06030B2
:10D29000301C000000181818180018181818000082
:10D2A00000E03030180C183030E000000073DACEA7
:10D2B000000000000000000000000010386CC6C62E
:10D2C000FE00000000000000000000000000000060
:10D2D000000000000000183C3C3C1818180018180A
:10D2E00000000000006666662400000000000000E8
:10D2F000000000000000006C6CFE6C6C6CFE6C6C3E
:10D300000000000018187CC6C2C07C060686C67CD9
:10D310001818000000000000C2C60C183060C68655
:10D32000000000000000386C6C3876DCCCCCCC7689
:10D3300000000000003030306000000000000000FD
:10D340000000000000000C18303030303030180C75
:10D3500000000000000030180C0C0C0C0C0C1830F5
:10D36000000000000000000000663CFF3C6600007A
:10D3700000000000000000000018187E18180000CF
:10D380000000000000000000000000000018181855
:10D390003000000000000000000000FE000000005F
:10D3A000000000000000000000000000000018184D
:10D3B000000000000000000002060C183060C08071
:10D3C000000000000000386CC6C6C6C6C6C66C3871
:10D3D0000000000000001838781818181818187E77
:10D3E0000000000000007CC6060C183060C0C6FEBD
:10D3F0000000000000007CC606063C060606C67C4F
:10D400000000000000000C1C3C6CCCFE0C0C0C1E40
:10D41000000000000000FEC0C0C0FC060606C67C7E
:10D420000000000000003860C0C0FCC6C6C6C67C54
:10D43000000000000000FEC606060C183030303038
:10D440000000000000007CC6C6C67CC6C6C6C67CFE
:10D450000000000000007CC6C6C67E0606060C78EA
:10D46000000000000000000018180000001818005C
:10D47000000000000000000018180000001818301C
:10D4800000000000000000060C18306030180C0688
:10D490000000000000000000007E00007E00000090
:10D4A000000000000000006030180C060C1830600E
:10D4B0000000000000007CC6C60C181818001818E0
:10D4C000000000000000007CC6C6DEDEDEDCC07CA2
:10D4D00000000000000010386CC6C6FEC6C6C6C6F6
:10D4E000000000000000FC6666667C66666666FCFE
:10D4F0000000000000003C66C2C0C0C0C0C2663C64
:10D50000000000000000F86C6666666666666CF8EF
:10D51000000000000000FE6662687868606266FED7
:10D52000000000000000FE6662687868606060F0DD
:10D530000000000000003C66C2C0C0DEC6C6663AFD
:10D54000000000000000C6C6C6C6FEC6C6C6C6C6E7
:10D550000000000000003C18181818181818183C93
:10D560000000000000001E0C0C0C0C0CCCCCCC7885
:10D57000000000000000E666666C78786C6666E67F
:10D58000000000000000F06060606060606266FEA5
:10D59000000000000000C6EEFEFED6C6C6C6C6C627
:10D5A000000000000000C6E6F6FEDECEC6C6C6C617
:10D5B0000000000000007CC6C6C6C6C6C6C6C67C43
:10D5C000000000000000FC6666667C60606060F041
:10D5D0000000000000007CC6C6C6C6C6C6D6DE7CFB
:10D5E0000C0E00000000FC6666667C6C666666E6F3
:10D5F0000000000000007CC6C660380C06C6C67C71
:10D600000000000000007E7E5A1818181818183CF8
:10D61000000000000000C6C6C6C6C6C6C6C6C67C98
:10D62000000000000000C6C6C6C6C6C6C66C3810DC
:10D63000000000000000C6C6C6C6D6D6D6FEEE6CF8
:10D64000000000000000C6C66C7C38387C6CC6C682
:10D65000000000000000666666663C181818183C5A
:10D66000000000000000FEC6860C183060C2C6FE36
:10D670000000000000003C30303030303030303CB2
:10D680000000000000000080C0E070381C0E0602A0
:10D690000000000000003C0C0C0C0C0C0C0C0C3CB2
:10D6A0000000000010386CC6000000000000000000
:10D6B000000000000000000000000000000000006A
:10D6C00000FF00000030180C000000000000000007
:10D6D000000000000000000000780C7CCCCCCC7670
:10D6E000000000000000E06060786C666666667CA2
:10D6F0000000000000000000007CC6C0C0C0C67C66
:10D700000000000000001C0C0C3C6CCCCCCCCC7697
:10D710000000000000000000007CC6FEC0C0C67C07
:10D720000000000000001C36323078303030307895
:10D7300000000000000000000076CCCCCCCCCC7CFB
:10D740000CCC78000000E060606C7666666666E689
:10D750000000000000001818003818181818183CAD
:10D760000000000000000606000E0606060606067B
:10D7700066663C000000E06060666C78786C66E687
:10D780000000000000003818181818181818183C65
:10D79000000000000000000000ECFED6D6D6D6C681
:10D7A000000000000000000000DC66666666666639
:10D7B0000000000000000000007CC6C6C6C6C67C93
:10D7C000000000000000000000DC66666666667C03
:10D7D0006060F000000000000076CCCCCCCCCC7CAB
:10D7E0000C0C1E000000000000DC7666606060F03B
:10D7F0000000000000000000007CC660380CC67C01
:10D80000000000000000103030FC30303030361C9A
:10D81000000000000000000000CCCCCCCCCCCC76CA
:10D82000000000000000000000C6C6C6C6C66C3876
:10D83000000000000000000000C6C6D6D6D6FE6C70
:10D84000000000000000000000C66C3838386CC6CC
:10D85000000000000000000000C6C6C6C6C6C67EA6
:10D86000060CF8000000000000FECC183060C6FE78
:10D870000000000000000E18181870181818180E74
:10D8800000000000000018181818181818181818A8
:10D89000000000000000701818180E1818181870F2
:10D8A000000000000076DC00000000000000000026
:10D8B0000000000000001C3000000000000000001C
:10D8C00000000000000070180000000000000000D0
:10D8D000000000000010386C000000000000000094
:10D8E0000000000000C6C6000000000000000000AC
:10D8F000000000000076DC000000000000000000D6
:10D900000000000000000000003818181818183C2B
:10D91000000000000000386C6C6C786C6666666C09
:10D9200060C00000102810007CC6C6FEC6C6C6C671
:10D93000000000000030483000780C7CCCCCCC7665
:10D940000000000000001E7AD8D8D8FED8D8DADE51
:10D95000000000000000FC666666F6F6666666FC7F
:10D96000000000000000F0607C666666667C60F087
:10D97000000000000000000000CC323E70B0B26C2D
:10D98000000000000000D060B0187CC6C6C6C67C8F
:10D99000000000000000E06060786C6C786060F06F
:10D9A0000000000000007CC6CECED6D6E6E6C67CDF
:10D9B0000000000000000000003A44CED6E644B863
:10D9C00000000000000000386CC6C6FEC6C6C6C611
:10D9D00000000000000000FE66626878686266FE73
:10D9E000000000000000003C181818181818183C17
:10D9F000000000000000007CC6C6C6C6C6C6C67CC5
:10DA000000000000000000C6C6C6C6C6C6C6C67C6A
:10DA100000000000000000C6E6F6FEDECEC6C6C668
:10DA20000000000000001818001818183C3C3C18B2
:10DA300000000000000030300030303060C6C67C8E
:10DA4000000000001C30000000000000000000008A
:10DA5000000000007018000000000000000000003E
:10DA600000000000386C0000000000000000000012
:10DA700000000000C6C6000000000000000000001A
:10DA80000000000076DC0000000000000000000044
:10DA90000000000000000000000000000000000086
:10DAA000183000000000000000000000000000002E
:10DAB0000000000000000010107CD0D0D0D0D67C38
:10DAC0001010000000001C30303078303030325CF4
:10DAD0000000000000000000423C24243C42000002
:10DAE000000000000000663C187E18187E18181808
:10DAF0000000000000001818181800001818181866
:10DB00000000000000003C6460384444380C4C784D
:10DB10000000000000C6C600000000000000000079
:10DB200000000000000000007E425A5E5A427E0063
:10DB30000000000000007008788888740000000071
:10DB4000000000000000000000366CD86C360000B9
:10DB50000000000000000000000000FC04040000C1
:10DB600000000000000000000000007C0000000039
:10DB700000000000000000007C4454444C547C0031
:10DB800000000000FE000000000000000000000097
:10DB9000000000000070D888D8700000000000006D
:10DBA000000000000000000010107C1010007C003D
:10DBB00000000000788C0C183060FC0000000000B1
:10DBC00000000000788C0C780C8C780000000000BD
:10DBD00000000000000E18200000000000000000FF
:10DBE0000000000000000000006666666666667C55
:10DBF0006060C00000007ED4D4D474141414143EA9
:10DC0000000000000000000000003838380000006C
:10DC10000000000060E060606060F0000000000054
:10DC20000000000000003C6666663C00000000004A
:10DC3000000000000000000000D86C366CD8000026
:10DC400000000000000040C0444810244C941E0412
:10DC500000000000000040C04448102C5284081E00
:10DC6000000000000000C0204428D0244C941E0472
:10DC7000000000000000000000663C183C66000048
:10DC800000000000000000001818007E00181800B6
:10DC90000000000000000000000818387FFF7F38F7
:10DCA00018080000000000000010181CFEFFFE1CF9
:10DCB0001810000000000000000010387CFE38380A
:10DCC0003838000000000000000038383838FE7C8A
:10DCD000381000000000000606060616367EFE7CA0
:10DCE00030100000000000000000030306060CCC0A
:10DCF0007838000000000000000000000000000074
:10DD00000000000000000000000000000000000013
:10DD10000000000000000000000000000000000003
:10DD20000000000000000000000000003800380083
:10DD3000380038003800380038003800380010004B
:10DD4000100000003800380038000000000000001B
:10DD500000000000000000000000000073807380DD
:10DD600073807380738000000000000000000000DA
:10DD700000000000000000000000000000000000A3
:10DD80000000000000000000000000000C600C60BB
:10DD90000C6018C0FFF0FFF018C039C03180FFF0F0
:10DDA000FFF031807380630063000000000000001A
:10DDB0000000000000000000000006001F803FC0BF
:10DDC00076E076E076007E003F001FC007E006E0C8
:10DDD00006E076E076E03FC01F8006000600000007
:10DDE0000000000000000000000000003C187E3829
:10DDF00066306630666066607EC03CC0019E01BFD2
:10DE000003B3033303330633063F0C1E0000000048
:10DE100000000000000000000000000007800FC0AC
:10DE20001CE01CE01EE00FC00F801F803F9C71FCB7
:10DE300071F870F079FC3FFE1F8C000000000000BC
:10DE400000000000000000000000000070007000F2
:10DE50007000700070000000000000000000000072
:10DE600000000000000000000000000000000000B2
:10DE70000000000000000000000000000C0018007E
:10DE800018003800380070007000700070007000DA
:10DE90007000700070003000380038001800180062
:10DEA0000C000000000000000000000060003000D6
:10DEB0003000380038001C001C001C001C001C0036
:10DEC0001C001C001C001800380038003000300016
:10DED00060000000000000000000000018001800B2
:10DEE000DB00FF001C003C00660024000000000076
:10DEF0000000000000000000000000000000000022
:10DF00000000000000000000000000000000000011
:10DF100007000700070007007FF07FF07FF0070091
:10DF200007000700070000000000000000000000DC
:10DF300000000000000000000000000000000000E1
:10DF400000000000000000000000000000000000D1
:10DF500000000000700070007000100030006000D1
:10DF600000000000000000000000000000000000B1
:10DF70000000000000000000000000007E007E00A5
:10DF80007E00000000000000000000000000000013
:10DF90000000000000000000000000000000000081
:10DFA0000000000000000000000000000000000071
:10DFB0000000000070007000700000000000000011
:10DFC0000000000000000000000000000C000C0039
:10DFD00018001800180038003000300030006000D1
:10DFE000600060006000C000C00000000000000091
:10DFF0000000000000000000000000000F003FC013
:10E0000039C070E070E070E070E070E070E070E0E7
:10E0100070E070E039C03FC00F0000000000000059
:10E0200000000000000000000000000003800380EA
:10E0300007801F803F803B80238003800380038014
:10E040000380038003800380038000000000000041
:10E050000000000000000000000000001F803FC022
:10E0600079E070E000E000E001C003C007800F002D
:10E070001E001C0038007FE07FE000000000000070
:10E080000000000000000000000000001F003F80B2
:10E0900071C071C001C003C00F800F8001C000E0DB
:10E0A00000E070E079C03FC01F00000000000000E9
:10E0B0000000000000000000000000000380078056
:10E0C00007800F800F801B80338033806380C38084
:10E0D000FFE0FFE0038003800380000000000000F9
:10E0E0000000000000000000000000001FC01FC072
:10E0F0003800380038003F807FC071E000E000E069
:10E1000000E070E079C03FC01F0000000000000088
:10E110000000000000000000000000000F803FC071
:10E1200039E07080700077807FC079C070E070E067
:10E1300070E070E039C03FC00F0000000000000038
:10E140000000000000000000000000007FE07FE011
:10E1500000E001C003800380070007000E000E00EE
:10E160000E001C001C001C001C0000000000000031
:10E170000000000000000000000000001F803FC001
:10E1800079E070E070E039C01F801F8039C070E016
:10E1900070E070E079E03FC01F80000000000000E8
:10E1A0000000000000000000000000000F003FC061
:10E1B00039C070E070E070E070E039E03FE01EE0F0
:10E1C00000E030E079C03FC01F0000000000000008
:10E1D000000000000000000000000000000000003F
:10E1E0000000000038003800380000000000000087
:10E1F0000000000038003800380000000000000077
:10E20000000000000000000000000000000000000E
:10E210000000000038003800380000000000000056
:10E2200000000000380038003800080018003000F6
:10E2300000000000000000000000000000000000DE
:10E24000002000E007E01F807C0070007E001FC0FF
:10E2500007E000E0002000000000000000000000D7
:10E2600000000000000000000000000000000000AE
:10E27000000000007FE07FE07FE0000000007FE022
:10E280007FE07FE0000000000000000000000000D0
:10E29000000000000000000000000000000000007E
:10E2A000400070007E001F8003E000E007E03F8038
:10E2B0007E00700040000000000000000000000030
:10E2C0000000000000000000000000000F803FE0A0
:10E2D00078F07070007000F001E003C00780070064
:10E2E0000700000007000700070000000000000012
:10E2F00000000000000000000000000003E007F044
:10E300000F1C1C0E19CE33E63666666666666666B8
:10E3100066666666666663FE31BE380E1C1C0F3C80
:10E3200007F003E0000000000000000007C007C085
:10E3300007C00EE00EE00EE01C701C7038383FF88D
:10E340003FF87FFC701C701CE00E00000000000015
:10E350000000000000000000000000003FE03FF06F
:10E360003FF83838383838383FF03FF03FF8381C3D
:10E37000381C381C3FFC3FF83FF000000000000054
:10E3800000000000000000000000000007C01FF0B7
:10E390003FF83C3C7818700070007000700070000E
:10E3A00078183C3C3FF81FF007C000000000000058
:10E3B0000000000000000000000000003FE03FF00F
:10E3C0003FF83838383C381C381C381C381C381C8E
:10E3D000381C38383FF83FF03FC000000000000014
:10E3E0000000000000000000000000003FF83FF8BF
:10E3F0003FF83800380038003FF03FF03FF0380079
:10E40000380038003FF83FF83FF8000000000000F7
:10E410000000000000000000000000003FF03FF09E
:10E420003FF03800380038003FE03FE03FE0380080
:10E4300038003800380038003800000000000000C4
:10E4400000000000000000000000000003E00FF8E2
:10E450001FFC3C1E780C7000700070FE70FE70FE99
:10E46000380E3C1E1FFE0FFC03E000000000000001
:10E47000000000000000000000000000703870384C
:10E4800070387038703870387FF87FF87FF87038DF
:10E490007038703870387038703800000000000034
:10E4A0000000000000000000000000000380038066
:10E4B0000380038003800380038003800380038044
:10E4C00003800380038003800380000000000000BD
:10E4D00000000000000000000000000001C001C0BA
:10E4E00001C001C001C001C001C001C001C0E1C044
:10E4F000E1C0F1C07FC07F801E000000000000006E
:10E50000000000000000000000000000383C3878E7
:10E5100038F038E039C03B803FC03FC03EE03CE0CF
:10E52000387038383838381C381C000000000000BB
:10E53000000000000000000000000000380038006B
:10E54000380038003800380038003800380038000B
:10E55000380038003FF03FF03FF0000000000000BE
:10E560000000000000000000000000007C1F7E3F53
:10E570007E3F763776377637777777777367736747
:10E5800073E773E773E771C771C70000000000000D
:10E590000000000000000000000000007038783823
:10E5A00078387C387E3876387738733873B871B8F5
:10E5B00071F870F870F87078703800000000000092
:10E5C00000000000000000000000000007E01FF84D
:10E5D0003FFC3C3C781E700E700E700E700E700E7C
:10E5E000781E3C3C3FFC1FF807E0000000000000E4
:10E5F0000000000000000000000000003FE03FF0CD
:10E600003FF83878383838783FF83FF03FE0380046
:10E6100038003800380038003800000000000000E2
:10E6200000000000000000000000000007E01FF8EC
:10E630003FFC3C3C781E700E700E700E700E708E9B
:10E6400079DE3CFC3FFC1FFE07EF000600000000E7
:10E650000000000000000000000000003FE03FF06C
:10E660003FF83838383838383FF83FF03FC038E0A6
:10E6700038F0387038383838381C00000000000096
:10E6800000000000000000000000000007C01FF0B4
:10E690003FF0387838383C001F800FF003F00078E6
:10E6A000703878783FF83FF00FC00000000000009D
:10E6B0000000000000000000000000007FF07FF07C
:10E6C0007FF00700070007000700070007000700AA
:10E6D0000700070007000700070000000000000017
:10E6E00000000000000000000000000070387038DA
:10E6F00070387038703870387038703870387038DA
:10E70000703878783FF03FF00FC000000000000044
:10E71000000000000000000000000000E038E07889
:10E7200070707070707038E038E038E01DC01DC047
:10E730001DC00F800F800F80070000000000000048
:10E74000000000000000000000000000E187E187F9
:10E75000718E718E718E718E399C399C399C399C69
:10E760001DB81DB81E781E781E781E7800000000A7
:10E770000000000000000000000000007038703849
:10E7800038701CE01CE00FC00780078007800FC0B6
:10E790001CE01CE038707038703800000000000089
:10E7A000000000000000000000000000E038E03839
:10E7B000707038E038E01DC00F800F800700070040
:10E7C0000700070007000700070000000000000026
:10E7D0000000000000000000000000007FF07FF05B
:10E7E0007FF000F001E003C007800F001E003C0036
:10E7F0007800F000FFF0FFF0FFF0000000000000E4
:10E800000000000000000000000000003E003E008C
:10E810003E00380038003800380038003800380032
:10E820003800380038003800380038003E003E001C
:10E830003E0000000000000000000000C000C0001A
:10E840006000600060006000300030003000380080
:10E850001800180018000C000C0000000000000058
:10E86000000000000000000000000000F800F800B8
:10E87000F800380038003800380038003800380018
:10E88000380038003800380038003800F800F80048
:10E89000F8000000000000000000000006000F006B
:10E8A0000F001F80198039C039C070E000000000DF
:10E8B0000000000000000000000000000000000058
:10E8C0000000000000000000000000000000000048
:10E8D0000000000000000000000000000000000038
:10E8E0000000000000000000000000000000FFF039
:10E8F000FFF000000000000000000000E0006000E9
:10E9000030000000000000000000000000000000D7
:10E9100000000000000000000000000000000000F7
:10E9200000000000000000000000000000000000E7
:10E93000000000001F803FC060E003E01FE03CE0FB
:10E9400070E070E071E03FE01E7000000000000029
:10E9500000000000000000000000000070007000D7
:10E960007000700077807FE078E070707070707079
:10E970007070707078E07FE0778000000000000029
:10E980000000000000000000000000000000000087
:10E99000000000000F003FC039C070E07000700040
:10E9A000700070E039C03FC00F00000000000000A0
:10E9B0000000000000000000000000000070007077
:10E9C000007000700F703FF038F0707070707070F1
:10E9D0007070707038F03FF00F70000000000000A1
:10E9E0000000000000000000000000000000000027
:10E9F000000000000F003FC039C070E07FE07FE002
:10EA0000700070E039C03FC00F000000000000003F
:10EA100000000000000000000000000000F001F015
:10EA2000038003803FFC3FFC03800380038003805E
:10EA30000380038003800380038000000000000047
:10EA400000000000000000000000000000000000C6
:10EA5000000000000F703FF038F070707070707040
:10EA60007070707038F03FF01F70007070F07FE0D1
:10EA70001FC00000000000000000000070007000D7
:10EA80007000700073C07FE078F07070707070700C
:10EA90007070707070707070707000000000000016
:10EAA0000000000000000000000000000380038060
:10EAB0000000000003800380038003800380038044
:10EAC00003800380038003800380000000000000B7
:10EAD0000000000000000000000000000380038030
:10EAE0000000000003800380038003800380038014
:10EAF000038003800380038003800380038007007A
:10EB00000E00000000000000000000007000700017
:10EB10007000700070E071C073807F007F007F0024
:10EB20007B80718071C070E070E000000000000028
:10EB300000000000000000000000000003800380CF
:10EB400003800380038003800380038003800380AD
:10EB50000380038003800380038000000000000026
:10EB600000000000000000000000000000000000A5
:10EB70000000000077CF7FFF71C771C771C771C7F1
:10EB800071C771C771C771C771C70000000000006D
:10EB90000000000000000000000000000000000075
:10EBA0000000000073C07FE078F0707070707070CB
:10EBB00070707070707070707070000000000000F5
:10EBC0000000000000000000000000000000000045
:10EBD000000000000F803FE038E0707070707070CF
:10EBE0007070707038E03FE00F800000000000009F
:10EBF0000000000000000000000000000000000015
:10EC00000000000077807FE078E0707070707070B6
:10EC10007070707078E07FE0778070007000700036
:10EC20007000000000000000000000000000000074
:10EC3000000000000F703FF038F07070707070705E
:10EC40007070707038F03FF00F70007000700070DE
:10EC50000070000000000000000000000000000044
:10EC600000000EFC0FFC03C00380038003800380C0
:10EC70000380038003800380038000000000000005
:10EC80000000000000000000000000000000000084
:10EC9000000000001F803FC070E070007E003FC099
:10ECA00007E000E070E03FC01F80000000000000AF
:10ECB00000000000000000000000000000000380D1
:10ECC000038003800FF00FF0038003800380038034
:10ECD00003800380038001F000F0000000000000CA
:10ECE0000000000000000000000000000000000024
:10ECF00000000000707070707070707070707070D4
:10ED00007070707078F03FF01F700000000000001D
:10ED100000000000000000000000000000000000F3
:10ED2000000000007070707038E038E038E01DC0FE
:10ED30001DC00F800F8007000700000000000000CA
:10ED400000000000000000000000000000000000C3
:10ED500000000000E38EE38E638C77DC76DC36D82F
:10ED600036D83EF83C781C701C7000000000000093
:10ED70000000000000000000000000000000000093
:10ED80000000000070E039C039C01F800F000F0084
:10ED90000F001F8039C039C070E000000000000083
:10EDA0000000000000000000000000000000000063
:10EDB00000000000E0E0E0E071C071C071803B80C5
:10EDC0003B801B001F001F000E000E001C007C007B
:10EDD00078000000000000000000000000000000BB
:10EDE000000000007FC07FC001C0038007000E004C
:10EDF0001C00380070007FC07FC0000000000000D1
:10EE000000000000000001000100400223C40FF0D8
:10EE10001FF81FF8DFFB1FF81FF80FF023C4400294
:10EE200001000100000000000000000000000000E0
:10EE30000000000000000000000000003000300072
:10EE40003000300030003000300030003000300042
:10EE50003000300030003000300030003000300032
:10EE600030003000000000800080000113C209F073
:10EE700000F80078187B007800F809F013C2000150
:10EE80000080008000000000000000000000000082
:10EE90000000000000000000000000000000000072
:10EEA00000000000000000007C20FFE0FFE087C0C1
:10EEB0000000000000000000000000000000000052
:10EEC0000000000008103030303830383038303032
:10EED0003078FCFC783000C1814001C0804101C025
:10EEE000804100C1814001C0804100C1814000C11A
:10EEF000814001C0804101C0804100C1814000C10A
:10EF0000814001C0804100C1814001C0804101C0F9
:10EF1000804100C1814001C0804100C1814000C1E9
:10EF2000814001C0804100C1814001C0804101C0D9
:10EF3000804100C1814000C1814001C0804101C0C9
:10EF4000804100C1814001C0804100C1814000C1B9
:10EF5000814001C0804101C0804100C1814000C1A9
:10EF6000814001C0804100C1814001C0804101C099
:10EF7000804100C1814000C1814001C0804101C089
:10EF8000804100C1814001C0804100C1814000C179
:10EF9000814001C0804100C1814001C0804101C069
:10EFA000804100C1814001C0804100C1814000C159
:10EFB000814001C0804101C0804100C1814000C149
:10EFC000814001C0804100C1814001C0804101C039
:10EFD000804100C1814000C0C101C30302C2C60616
:10EFE00007C705C5C404CC0C0DCD0FCFCE0E0ACA81
:10EFF000CB0BC90908C8D81819D91BDBDA1A1EDED1
:10F00000DF1FDD1D1CDC14D4D515D71716D6D21280
:10F0100013D311D1D010F03031F133F3F23236F690
:10F02000F737F53534F43CFCFD3DFF3F3EFEFA3A40
:10F030003BFB39F9F83828E8E929EB2B2AEAEE2ED0
:10F040002FEF2DEDEC2CE42425E527E7E62622E240
:10F05000E323E12120E0A06061A163A3A26266A690
:10F06000A767A56564A46CACAD6DAF6F6EAEAA6A00
:10F070006BAB69A9A86878B8B979BB7B7ABABE7E50
:10F080007FBF7DBDBC7CB47475B577B7B67672B200
:10F09000B373B17170B05090915193535292965690
:10F0A0005797559594549C5C5D9D5F9F9E5E5A9AC0
:10F0B0009B5B99595898884849894B8B8A4A4E8E50
:10F0C0008F4F8D4D4C8C44848545874746868242C0
:10F0D00043834181804054532D3220564552203283
:10F0E0002E3800000000000004FA97999999D93F42
:10F0F000AF788E1DC571CC3F9FC678D0099AC33FAB
:10F10000935555555555E53F599322942449D23F7F
:10F11000DE03CB966446C73F44523EDF12F1C23F46
:10F12000000000000000000048F10008000000207E
:10F13000A000000028710008E8F10008A0000020ED
:10F1400000170000447100080000000000000000EB
:10F15000000000000000010203040102030406078E
:10F16000080902040608000000000000000000007A
:10F17000000000000000000000000000000000008F
:10F18000000000000000000000000000000000007F
:10F19000000000000000000000000000000000006F
:10F1A000000000000000000000000000000000005F
:10F1B000000000000000000000000000000000004F
:10F1C000000000000000000000000000000000003F
:10F1D0000000000000A24A0400000000000000003F
:08F1E0000102030406070809FF
:04000005080070ED92
:00000001FF
